:100000000C9400010C9400000C9400000C9400006F
:100010000C9400000C9400000C9400000C94000060
:100020000C9400000C9400000C9400000C94000050
:100030000C9400000C9400000C9400000C94000040
:100040000C9462010C9400000C942F010C9400009D
:100050000C9400000C9400000C9400000C94000020
:100060000C9400000C9400001027E80364000A00C0
:1000700001000010000110000100000000000A0053
:10008000320050001E0023003200640032000A00DB
:1000900001000A0001000F006400640064000A000F
:1000A00001000200010024003200FF00FF001E00DA
:1000B000140014001400E8032201C4097E02B400F5
:1000C0004200A4018403E8030000000000000000D7
:1000D0000000000000000000000000000000000020
:1000E0000000000000000000000000000000000010
:1000F0000000000000000000000000000000000000
:10010000000000000A0A0A0A0A0A0A0A0A0A0A0A77
:100110000A0A0A0A020002007A00020004007C00B7
:10012000010007037E0001000C04800001000D04A3
:10013000820001000E04840001000F04860001000B
:1001400010048800010011048A00010013048C00CF
:10015000010014048E0001001904900001001A042B
:10016000920001001B04940001001C049600010091
:100170001D04980001001E049A0001001F049C0049
:10018000010021049E0001002204A00001002304BC
:10019000A20001002C04A40001002F04A60001000D
:1001A0003804A80001003A04AA0001003B04AC0096
:1001B00001003C04AE0001003D04B00001003E041B
:1001C000B20001003F04B40002004404B600020083
:1001D0004804B80002004A04BA0002004E04BC0001
:1001E00001005004BE0001005204C0000200580487
:1001F000C20002005A04C40002005C04C6000000F1
:10020000F894EE27EFBBF1E0F5BFE5BF8DE0A2E08B
:10021000BB27ED938A95E9F780E098E0A0E0B1E094
:10022000ED930197E9F7E4E1F1E08591959100976D
:1002300061F0A591B59105901590BF01F001059071
:100240000D920197E1F7FB01F0CFE8E0EEBBEFEF95
:10025000EDBFE8E0EEBFC0E0D3E00C947804AA93D1
:10026000EA93FA93EFB7EA931A930A931091C000B6
:100270000091C600E12FEC71E9F4E0918704EF5F93
:10028000E0938704E150F0E0E259FB4F0083A09136
:100290008704A93119F4E0E0E0938704A091890470
:1002A000AF5FA0938904A93129F4E0E0E0938904C9
:1002B000689437F809911991E991EFBFF991E991A3
:1002C000A99118950A921A926A937A938A939A93AB
:1002D000AA93BA93EA93FA93EFB7EA93E09155039E
:1002E000F09156033196E0935503F09356030E9424
:1002F000FE30E1E5F1E00E941F3E0E2E0E94FE302E
:10030000E3EAF2E00E941F3EE02909F434C2A09122
:100310005303B0915403E5E0F0E00E94433E0E2EFB
:10032000A0912903EEE00E94153EE02121F0E0912A
:100330002903EF5F03C025FC03C0E0E0E09329033D
:10034000A0912903AE3011F4689425F8A0913203EE
:10035000A13029F4F79B02C0F79801C0F79AE1E0B9
:100360002E260E9403310E940C31E093EB03F093A0
:10037000EC036093ED037093EE030E941331AFEC36
:10038000B3E00E9418310E941F31ABEFB3E00E942E
:1003900018310E9424310E942D310E94463DE09385
:1003A000CF03F093D0036093D1037093D203A09155
:1003B000FB03B091FC038091FD039091FE03E0E00C
:1003C000F0E060E772E40E94463DE093FB03F093A7
:1003D000FC036093FD037093FE030E9432310E9480
:1003E00037310E2E0E943C310E943731E02161F1FD
:1003F000E091FB03F091FC036091FD037091FE031B
:100400000E9424310E94463DE093F703F093F803E5
:100410006093F9037093FA030E944131A7E6B3E0B9
:100420000E944A31A091F703B091F8038091F9033B
:100430009091FA030E940C31E093D703F093D80314
:100440006093D9037093DA030E944F310E945831B0
:100450000E9461310E94A83CE093DF03F093E00327
:100460006093E1037093E2030E944F310E946A316E
:100470000E94AB3D0E2E0E946F31E8EEFDEF0E9410
:100480003D3EE021D1F00E944F310E945831A091B1
:100490000304B091040480910504909106040E9425
:1004A0007431E0930304F0930404609305047093A3
:1004B0000604A5E7B3E00E944A310E944F310E9432
:1004C00058310E9479310E94A83CE0930704F093D0
:1004D00008046093090470930A040E9482310E9408
:1004E0008B310E947431A7EBB3E00E94373C0E942D
:1004F000313F0E948231AAE0B0E080E090E00E94AB
:10050000713E0E9479310E946C3C0E948B3D70F0DC
:10051000E0E0E0930704E0930804E0930904E0932B
:100520000A040E949E3131960E94A331E091BB03E0
:10053000F091BC036091BD037091BE030E944F31E6
:100540000E94F83CDF01CB010E940C31E093EF03E5
:10055000F093F0036093F1037093F2030E94A831CB
:100560000E94A83C0E94B131E0910E03F0E00E948D
:10057000BA310E94ED3D0E94C331A9E8B3E00E9468
:10058000D2310E9403310E945C3F3CF5A091EF0301
:10059000B091F0038091F1039091F2030E94D73162
:1005A0007F936F93FF93EF93A091EB03B091EC03D4
:1005B0008091ED039091EE030E94D731AF91BF91EE
:1005C0008F919F910E94463DE093E703F093E803EB
:1005D0006093E9037093EA0309C0E0E0E093E70366
:1005E000E093E803E093E903E093EA03A091EA03D0
:1005F000AA238AF40E94DE310E94E73118F40E9497
:10060000EE3108C00E94F5310E94023CA1E9B3E03E
:100610000E94D23114C00E94DE31E0E0F0EC69E7C4
:1006200074E40E948B3D09F008F403C00E94EE318F
:1006300006C00E94F531A1E9B3E00E94D2310E94C8
:10064000FE310E9407320E94A83C0E941032E091C5
:10065000CF03F091D0036091D1037091D2030E9437
:1006600019320E948B3D68F5E091D703F091D803D1
:100670006091D9037091DA030E9419320E94A83C5C
:10068000E093D303F093D4036093D5037093D60320
:100690000E9419320E9422320E94A13CDF01CB014C
:1006A0000E9441310E94463DA0E0B0E081E695E421
:1006B0000E94F83CA5E8B3E00E94D231689424F887
:1006C00002C0E0E12E260E94FE310E942B320E94E1
:1006D000A83CE093DB03F093DC036093DD037093AD
:1006E000DE030E942B32E0E0F0E060E87FE30E944E
:1006F0008B3D09F008F412C0E093DB03E093DC03C8
:10070000E093DD03E093DE030E943432EF5FFF4F9E
:100710006F4F7F4F0E943D320E9446320E945032FE
:10072000A034E2E4BE07EFE08E07E0E09E0788F029
:10073000E0E0E0937703E0937803E0937903E093BC
:100740007A03E0936A04E0936B04E0936C04E09313
:100750006D040E9407320E945932A7E5B3E00E945F
:100760004A31A0912703AC3308F4F298A0912703F3
:10077000AC3309F4F29A0E94FE30A33AE2E0BE07DD
:1007800009F08DC0A09126030E945D320E94623262
:100790000E946A310E94493E0E946B32E02191F032
:1007A000E0912703EF5FE0932703E0912603F0E059
:1007B0003296A0912703B0E0EA17FB0719F4ECE3A7
:1007C000E0932703E0E0E0935503E0935603D394CE
:1007D000A0910F03A13028F4E0910F03EF5FE093A5
:1007E0000F030E947232E8E5F2E00E943D3E0E2EB9
:1007F0000E947732E02199F0E0916B03F0916C0355
:100800003196E0936B03F0936C030E9472320E9466
:100810007C32EA1BFB0BE0937103F0937203ECE371
:10082000ED1589F4DD24C394EC1569F4CC24E09132
:100830000003EF5FE0930003A0910003A43119F4DB
:10084000E0E0E0930003A0912E03A130D0F0E0910E
:100850001203EF5FE0931203A0911203A23088F01D
:10086000E0911103EF5FE0931103E0E0E0931203E6
:10087000E0912E03A0911103EA1718F4E0E0E09351
:100880001103E0912E03E03019F4E0E0E09311034E
:10089000A0912E03A23019F4E1E0E0931103E99155
:1008A000EFBFF991E991B991A991999189917991C4
:1008B0006991199009901895AA93E881E066E093F0
:1008C0007C0085E28A95F1F7E0917A00E064E0939C
:1008D0007A00E0917A00E071E1F3E0917A00E06162
:1008E000E0937A00E0917800F091790021960895E4
:1008F000EF9763978CE4A6E0B0E0E8ECF0E00E94AC
:10090000713FFF2411E001E0E0E8E0936100E0E0E6
:10091000E0936100EFE0E4B9E1E0E5B9E0E0E7B9D8
:10092000E4E0E8B9EAEFEAB9E7EEEBB9E0E0E4BD0C
:10093000E3E0E5BDE0E0E6BDE7BDE8BDE0938000B3
:10094000E0938100E0938500E0938400E0938700CA
:10095000E0938600E0938900E0938800E0938B00A9
:10096000E0938A00E093B600E1EAE093B000E2E0B1
:10097000E093B100E0E0E093B200E093B300E093D5
:10098000B400E1E0E0936E00E0E0E0936F00E093FC
:100990007000E0936900EDBBE0936800E093C00055
:1009A000E8E9E093C100E6E0E093C200E0E0E09314
:1009B000C500E7E4E093C400E0E8E0BFE0E0E093D6
:1009C0007F00E0937E00E0E6E0937C00E6E2E093C7
:1009D0007A00E0E0E0937B00ECBDE093BC0078940B
:1009E0005F9A0E9481320E9485320E948B320E945F
:1009F00092320E949F320E948132EAE06E1670F5B8
:100A0000E0E0E0934604E0934704E0933104E09390
:100A10003204E0934104E0934204E0934304E8EE9F
:100A2000F3E0E0935C04F0935D04E0E0E0935E04A7
:100A3000E0935F04E0936004E0936104E093620458
:100A4000E0936304E0936404E0936504E093660438
:100A5000E0936704E0936804E0936904EAE09E167B
:100A600058F4E0E0E0934C04E0934D04E093540428
:100A7000E0935504689426F8EAE0BE1618F46894EA
:100A800030F827F8689433F8E9E1E09316030E9400
:100A9000AC32E8ECF0E00E94B332E0EDF7E00E9407
:100AA000B832E8ECF0E0E0937F03F0938003E0914C
:100AB0000B04E0931703E0910C04E0931803E0911A
:100AC0000D04E0931903E0910E04E0931B03E09101
:100AD0000F04ECA7E0911004EDA7E0911104EEA73C
:100AE000E0911204E0931C03E0911304E0931D03D2
:100AF000F798F198E0911504E0932603E0914404FF
:100B0000F09145040E94BD32E0911D04E8A7E091F8
:100B10001E04E9A7E0911F04EAA7E0911604ECA3E4
:100B2000E0911704EDA3E0911804EEA3E0914804CE
:100B3000F0914904EB8BFC8BE0911904E0933303B3
:100B4000E0911A04E0933503E0911B04E093340331
:100B5000E0916A04F0916B0460916C0470916D04F3
:100B60000E943D32E0914604F0914704ABECB3E0C3
:100B70000E9418310E942232A7E5B3E00E944A3158
:100B80000E9407320E94C2320E941032E0911C047F
:100B9000F0E0EB87FC87E0914A04F0914B04EF8B87
:100BA000F88FE0915A04F0915B04ED87FE87E091A5
:100BB0004C04F0914D04AFEDB3E00E941831E09188
:100BC0005404F0915504AFEFB3E00E9418310E9435
:100BD000A8310E94C2320E94B131E0914E04F091DE
:100BE0004F040E94C632E0915204F09153046627EC
:100BF00077270E94CB32E09120040E946C3F23F8BB
:100C0000E0915004F09151040E94D432E09121040B
:100C1000E0930603E0912204E0930803E0912304AB
:100C2000E0930903E0912404E0930A03E091250492
:100C3000E0930B03E0912604E0930C03E09127047A
:100C4000E0932A03E0912804E0932B03E091290428
:100C5000E0932C03E0912A04E0932D03E0912B0410
:100C6000E0932E03E0912C04E0932F03E0912D04F8
:100C7000E0933003E0912E04E0933103E0915604B9
:100C8000F09157040E94A331E0912F04E0930E03EA
:100C9000E09130040E946C3F36F8E0913304E09319
:100CA0001003E0913404EF8FE0915804F09159045F
:100CB000EF87F88BE0913504E0934103E09136042F
:100CC000E0934203E0913704E0934303E09138045A
:100CD000E0931E03E0913904E0932003E0911404B3
:100CE000E0932103E0913A04E0932203E0913B0476
:100CF000E0932303E0913C04E0931503E0913D046D
:100D0000E0934A03E0913E04E0934B03E0913F04FB
:100D1000E0934C03E0914004E0934E03E0916804BB
:100D2000F0916904E0937503F0937603E091680411
:100D3000F0916904A3E0B4E00E94183136FE06C0C9
:100D4000C0903104E0913204E0930003E1E0E093CD
:100D50003F03A0910203AE3128F4E0910203EF5F5C
:100D6000E0930203A0910203AE3189F4E0E0E09346
:100D70003803E0939903E0939A03EBE0F0E00E94DC
:100D8000D932E8EB0E94DE32E4E1E0930203EF8D1A
:100D9000E03041F5A0916E04ECE30E94F73D0E2E89
:100DA000A0916F04E7E00E94F73D0E22A091870416
:100DB000EBE00E94F73DE02169F0E0917004E093E0
:100DC0003703E0917104E09338030E94E432E0E0DD
:100DD000E0930203A0918704AC3020F00E94F2322D
:100DE0000E94FE32AF8DA130D1F4A0916E04E8E2F2
:100DF0000E94F73D0E2EA0918704E8E00E94F73D87
:100E0000E02129F00E94E432E0E0E0930203A091A7
:100E10008704AC3020F00E94F2320E94FE32AF8D87
:100E2000A33009F079C0A0916E04ECE60E94F73D72
:100E30000E2EA0916F04EBE00E94F73D0E22A091D0
:100E40008704EFE00E94F73DE02109F441C0E09102
:100E50007104E0933703E0917204E0933803E0916A
:100E60007304F0E00E940A33F0919903E0E00E94DD
:100E70000A33E0917404F0E0A0919903B0919A03D1
:100E8000EA0FFB1F0E940A33E0917504E0934803C8
:100E9000E0917804E0934703E0917904F0E00E9448
:100EA000D932E0917A04E0933903E0917604F0E0DE
:100EB000E0939B03F0939C03E0917704F0E0E093D0
:100EC0009D03F0939E03E0E0E0938704E093020328
:100ED000A0918704A03100F1E0E0E0936E04E0937C
:100EE0006F04E0937004E0937104E0937204E09364
:100EF0007304E0937404E0937504E0937604E09344
:100F00007704E0937804EBE0E0937904E8EBE09376
:100F10007A04E0E0E0938704E8EC5E1630F4539442
:100F2000EEE1E51511F4E1E04E2E0E940F33E7EA01
:100F3000E0937A00A6E00E941333EF83F887E7E29C
:100F4000E0937A000E940F330E9485320E94E23DB6
:100F50000E94DE3DE987FA87E7E2E0937A000E948B
:100F60000F330E941A333B97A0F1A0E00E94133385
:100F7000662777270E942333A8EEB3E080E090E055
:100F80000E949C3EDF01CB010E942C33662777270D
:100F90000E94DE3E0E942333ABEBB3E00E946E3C26
:100FA0000E94313FE0910703EF5FE0930703E09178
:100FB0000603A0910703AE1750F00E943133E0936F
:100FC000B303F093B4036093B5037093B603E8944E
:100FD000F3F80E943A330E9485320E948B320E94BD
:100FE0004133A2E00E941333DF01E5E0F0E00E940C
:100FF000A13E8E2E0E943A330E949F328AE48A9547
:10100000F1F70E9492320E9441330E9448330E94BD
:101010003A33E7EAE0937A00A5E04EDCEF2FF0E008
:10102000E98FFA8F0E943A330E941A33AE2E0E9443
:101030003A33A0914E03A13069F4E98DFA8DA98D60
:10104000BA8D0E94693EDF01E6EDF0E00E94A13E0C
:10105000E98FFA8FE0911003E03009F0A0C0E1E0E1
:10106000E515B1F50E9452335E9710F4E1E0EAA372
:101070000E9452330E9457330E945233EAEFF0E04D
:101080000E943D3EE02111F0E2E0EAA30E945233CB
:10109000AB3FE0E0BE0710F0E3E0EAA3A98DBA8D14
:1010A0005E9710F4E1E0E9A30E945D33A98DBA8D4B
:1010B000EAEFF0E00E943D3EE02111F0E2E0E9A31A
:1010C000A98DBA8DAB3FE0E0BE0710F0E3E0E9A3E5
:1010D0000E9452330E946033AAA10E946B3311F028
:1010E000E4E009C00E9452330E947033AAA10E941A
:1010F0006B3311F0E5E0EAA3A98DBA8D0E9460334D
:10110000A9A10E946B3311F0E4E009C0A98DBA8D4A
:101110000E947033A9A10E946B3311F0E5E0E9A3AE
:10112000AAA10E945D32AAA10E947B3369F0E98DD9
:10113000FA8D0E948033E8E2F0E0E98FFA8FAE8109
:10114000AC3511F40E948533AAA10E948B33AAA169
:10115000E5E00E94F73DE02911F00E948533A9A146
:101160000E945D32A9A10E947B3369F0E8E2F0E0C1
:10117000E98FFA8FAAA10E945D32AAA10E947B3357
:1011800011F00E948533A9A10E948B330E949033F5
:10119000E02921F0ECE3F0E0E98FFA8F03C0E0E012
:1011A000EAA3E9A3A98DBA8DA73DE0E0BE0720F030
:1011B000E6EDF0E0E98FFA8F0E9495330E949B33B1
:1011C0000E94153EE021E9F1E4E1ED8F6894F3F827
:1011D0000E94A5330E94AB3319F0E1E0E0931403C1
:1011E000A12F0E94B4330E94B93321F0F398F49AEE
:1011F00012E01CC0A12FE2E00E94F73D0E2E0E94DB
:10120000B93359F0F498F59AAEA5A13010F013E077
:1012100003C0F598F39A11E009C0A12F0E94BC33D6
:101220000E94B93319F0F598F39A11E0A62DE9E080
:101230000E941A3E0E2E0E94AB3319F0E0E0E093BC
:101240001403E0914F03E09340030E945233D3977D
:1012500008F45DC00E94C1330E94C633E12F0E9492
:10126000CD3320F0E8ECF0E00E948033A0914203FF
:10127000A13011F40E94DD33E12F0E94E8330E9477
:10128000F833AC91A13008F441C00E94FF330E94B2
:1012900008340E94673F4CF40E94F8330E941434D3
:1012A0000E94B73D0E941E3423C00E9427340E9432
:1012B0002934EF930E9427340E943234AF91EA23FD
:1012C00079F00E94F8330E9414340E94BC3DA09330
:1012D000A303B093A4038093A5039093A60308C02F
:1012E0000E9427340E943B341CF00E9445340EC0FB
:1012F000A091A303B091A4038091A5039091A603AC
:101300000E9454340E94DE3E0E94803304C00E943A
:1013100085330E9445340E94A5330E9459340E2221
:101320000E945E3401F10E9452330E94583F10F433
:10133000E4E1EB8FA09128030E945D320E946234A9
:10134000E02141F0E3E0E0933603E0E0E09328039E
:101350000E946834E0914F03E09328036894F0F80A
:1013600021F8E894F4F8A0913003A130D9F50E9457
:101370006E340E2EA0914003E0E50E94153E0E2231
:10138000A0912803E8EC0E94153E0E9470340E22C2
:10139000A0E0F4FCA1E00E94783429F0E091280359
:1013A000EF5FE09328030E945D33A98DBA8DE0E5DD
:1013B000F0E00E943D3E0E22A0912803E0E00E9452
:1013C0001A3E0E947034E02169F0E0912803E15058
:1013D000E09328030E947D340E94813419F0E3E0F9
:1013E0000E9487340E9462340E948A34A0912803AC
:1013F0000E946B3321F0E0E0E093290306C0A09146
:101400002903A23010F4E89425F8A0912803A13014
:1014100020F0E0912803F0E002C00E94C133E09385
:101420005303F09354030E94C133309729F4E89496
:1014300021F86894F4F827C00E9493340E2E0E947D
:101440006E340E22A09130030E946B331E2EA091A9
:1014500028030E945D320E9493340E22A091400323
:10146000EFE40E941A3E0E22A09130030E947834CD
:10147000E12949F0E0E0E09328030E948533E894F5
:1014800022F8689421F8E09104030E945233F0E0BE
:10149000EA17FB0720F4E0914F03E09304030E9456
:1014A0009A340E94613E0E22A09133030E946B3356
:1014B0001E2E0E949A340E94593E0E22A09134039F
:1014C0000E946B33E12961F0E0914F03E093040344
:1014D0000E947D340E94A93419F0E2E00E94873412
:1014E000A0912803A13080F0689422F80E94C133B3
:1014F000A0912803B0E0AE17BF0728F0E0912803C1
:10150000F0E00E94803302C0E89422F80E94AD34DB
:101510000E22A0E031FCA1E00E946B3331F0689410
:1015200031F80E94C1330E94B3320E94AD34E021F1
:1015300061F10E94C3340E94CB34A4F0A091AF03A8
:10154000B091B003EB89FC89EA1BFB0BA3E0B0E090
:101550000E94973E0E94D334AE1BBF0BA093810321
:10156000B09382030E94C3340E945C3F2CF40E941B
:10157000D83432970E94B332A0918203AA232AF46E
:10158000E0E0E0938103E09382030E94DD340E9457
:10159000623F84F50E94DD340E94BC3D0E94CB3442
:1015A00074F0AB89BC89E091AF03F091B003EA1B02
:1015B000FB0B0E94D334EA0FFB1F0E94B3320E9440
:1015C000DD340E94BC3DA230E0E0BE07E0E08E07C3
:1015D000E0E09E072CF00E94D83431960E94B3328E
:1015E0000E94D334AB3FE0E0BE0724F0EAEFF0E026
:1015F0000E94B3320E94D8340E945233AE17BF0704
:1016000010F4E89431F80E94D8340E945233EA175B
:10161000FB0720F40E94D8340E9480330E94EA34F1
:10162000A0E032FCA1E00E94FC340E94813431F041
:10163000689432F80E9401350E94B8320E94EA3460
:101640000E948134A1F10E940635DF01CB01E0E068
:10165000F0E060E070E40E948B3D09F008F414C0F3
:101660000E940635A0E0B0E080E890E40E94F83CDB
:101670000E9415350E94F23D0E94423F0E94743143
:10168000A3E8B3E00E94D2310E9406350E94523F87
:101690002CF40E941A3535970E94B832A091840329
:1016A000AA232AF4E0E0E0938303E0938403EB852C
:1016B000FC850E941F350E9428350E94AB3D0E2EEE
:1016C0000E948134A9F10E942D35DF01CB01E0E0B9
:1016D000F0E060E470E40E948B3D09F008F414C06F
:1016E0000E942D35A0E0B0E080EA90E40E94F83C32
:1016F000DF01CB010E941A350E943C350E94A83CB4
:10170000A3E8B3E00E94D2310E942D350E94523FDF
:101710002CF40E941A3535960E94B8320E94153575
:10172000A53CE9E0BE0724F0E4ECF9E00E94B83201
:101730000E940135DF010E941A350E943D3E0E2EA7
:101740000E94813411F0E89432F80E940135DF01E3
:101750000E941A350E94433E0E2E0E94813421F0D1
:101760000E9415350E9441350E9446350E94613E17
:101770000E2EA0E034FCA1E00E946B3331F068949F
:1017800034F80E9401350E944D350E9446350E9472
:10179000623F5CF50E9452350E94CB349CF0E09190
:1017A0001803F0E0A091AB03B091AC03AE1BBF0BEC
:1017B000E3E0F0E00E945B35AE1BBF0BA0938B0310
:1017C000B0938C030E9452350E945C3F2CF40E941F
:1017D000623532970E944D35A0918C03AA232AF4DA
:1017E000E0E0E0938B03E0938C030E9446350E9477
:1017F000673F8CF50E946735A430E0E0BE07E0E06B
:101800008E07E0E09E078CF0A0911803BB27E091C3
:10181000AB03F091AC03AE1BBF0BE2E0F0E00E9423
:101820005B35EA0FFB1F0E944D350E9467350E9411
:101830005C3F2CF40E94623532960E944D35A09197
:101840008B03B0918C03A53CE9E0BE0724F0E4ECE7
:10185000F9E00E944D350E940135DF010E9462359A
:10186000AE17BF0710F4E89434F80E940135DF0189
:101870000E946235EA17FB0730F4A0918B03B09108
:101880008C030E944135E09113030E945233F0E033
:10189000EA17FB0720F4E0914F03E0931303E09174
:1018A0001303F0E035970E9452330E943D3E6E2FA5
:1018B0000E2EA0E031FCA1E00E9478341E2E062EF0
:1018C000A0E032FCA1E00E9478341E2A062EA0E09F
:1018D00034FCA1E00E947834E12961F0E0914F03EB
:1018E000E09313030E947D340E94813419F0E2E0FA
:1018F0000E948734A0913603A13078F00E9485338E
:10190000A0913603A13021F4EAE0F0E00E94803398
:10191000E0913603E150E09336030E945D33A091DD
:1019200030030E946B331E2EA98DBA8DE0E5F0E0E6
:101930000E94433E0E2EA0913003E1E00E94F73D4D
:101940000E947034E0211E2A0E945D33A091300372
:10195000E1E00E94F73D0E220E94A934E129E9F05E
:10196000E0E0E0930503A0912803A13018F0E2E045
:10197000E0933603E0E0E0932803E98DFA8DF297D7
:101980000E942835A6EFB8E28CE99FE30E94F83C5C
:10199000DE0159960E944A3103C0E0E0E98FEA8FE8
:1019A0000E94C133E98BFA8B0E9477350E2EA091ED
:1019B0002B030E94783411F0299A01C029980E94C3
:1019C00077350E2EA0914103E2E00E94F73DE02121
:1019D00011F0EFEF01C0E0E0E09344030E94A53373
:1019E0000E945934E02119F0E98DE0934D03A09154
:1019F0004D03A13068F0E0914D03F0E0E98FFA8FDC
:101A00000E9452330E94583F18F4E0E0E0934D03E7
:101A1000A82DE4E60E94153E6E2F0E2E0E947A3508
:101A20000E22AE81EDE50E94FC3D0E9481351E2E06
:101A3000062E0E947A350E220E945934E0211E2A79
:101A40000E947C320E9472320E941F3E0E948835A2
:101A50000E947732E021E12999F1E0915703F0915A
:101A60005803E0934604F09347040E9490350E9487
:101A700094350E9490350E94A8310E945932A4E505
:101A8000B4E00E944A310E9490350E949F35C09276
:101A900031040E949035E0910003E09332040E94EB
:101AA00090350E94A535E0936804F09369040E9484
:101AB00081325F98A8EEB3E00E94F83B5F98FECFBA
:101AC000AB2D0E94AA350E945934E02131F0E894F0
:101AD000F2F827F8E0E0E0933D030E94AF350E9462
:101AE0005934E02171F0E0913D03EF5FE0933D0355
:101AF000A0913D03AA3029F4E0E0E0933D03E09398
:101B000032030E94AF35A0E0F2FCA1E00E94FC3459
:101B10000E945934E021C1F1E4E1EC8F6894F2F8BD
:101B2000E0913203EF5FE0933203A09132030E9411
:101B3000BC330E945E3419F0E1E0E0933203A091DF
:101B400032030E948B330E945E3419F0E2E0E0938E
:101B50003203A09132030E94BC33A0912B030E9458
:101B6000FC340E94813419F0E1E0E0933203A0914B
:101B700032030E948B33A0E0F0FCA1E00E94783495
:101B800019F0E3E0E0933203E0913203E03031F406
:101B9000F7982A98E0E0E09345031EC0A091320335
:101BA000A13031F42A98EFEFE0934503E0E014C050
:101BB000A0913203A23039F4F79A2A98EFEFE0931C
:101BC0004503E0E009C0A0913203A33039F4F79A4D
:101BD0002A9AEFEFE0934503E09346030E94B8355D
:101BE000E081E093B4000E946E340E2E0E9477359F
:101BF0000E220E94A93429F1A0912A03A13009F4F0
:101C00005C9AE0910303EF5FE0930303A091030369
:101C1000E5E00E941A3E0E2EE4E10E94153EE0210E
:101C200041F0E0910303E170AFEFEA02F001E093CD
:101C3000B400A0910303A03118F0E0E0E0930303A7
:101C400025C05C98A0E030FCA1E00E94B433A091D4
:101C500032030E946B33D1F0E0913C03EF5FE093DD
:101C60003C03A0913C03A13019F4EFEFE093B400E2
:101C7000A0913C03A33019F4E0E0E093B400A091FC
:101C80003C03A43019F4E0E0E0933C030E94BE352D
:101C90000E94C535E1F0E0911D03A0911F03AE172E
:101CA00028F4E0911F03EE5FE0931F03E0911D0312
:101CB000A0911F03EA1728F4E0911F03E250E0937C
:101CC0001F03033621F4E0911D03E0931F030E94DC
:101CD000BE35EA17FB07E0F4E0911E03A0911F0355
:101CE000AE1728F4E0911F03EE5FE0931F03E0912D
:101CF0001E03A0911F03EA1728F4E0911F03E2508E
:101D0000E0931F03033621F4E0911E03E0931F03C9
:101D1000E0911F03E093B300EAE0E91518F4E894BA
:101D2000F1F826F80E94CE35A0E026FCA1E00E9442
:101D3000FC34A0E0F1FCA1E00E94FC340E94593484
:101D4000E02139F16894F1F8E0910D03EF5FE09341
:101D50000D03E0E0E8A3A8A1A53088F40E94D435E3
:101D6000A081A13018F0E5E0E8A305C0E0910D03E3
:101D7000EF5FE0930D03E8A1EF5FE8A3ECCFA09144
:101D80000D03A53018F0E0E0E0930D030E94D43578
:101D900000810E94CE35A0912503EFEF0E94153EF1
:101DA000E02121F0E0912503EF5F03C0E894F1F812
:101DB000E0E0E0932503A0912503A43109F099C147
:101DC000AE81E0E00E940B3E0E2E0E945934E021CD
:101DD00019F0EE81E150EE83033610F403E689C179
:101DE00001E0E0E0E0930D03E0911703E0930B04C2
:101DF0000E949035E0911803E0930C040E94903506
:101E0000E0911903E0930D040E949035E0911B03CB
:101E1000E0930E040E949035ECA5E0930F040E941D
:101E20009035EDA5E09310040E949035EEA5E09367
:101E300011040E949035E0911C03E09312040E946B
:101E40009035E0911D03E09313040E949035E091DA
:101E50002103E09314040E949035E0912603E0935F
:101E600015040E9490350E942C33E0934404F093B3
:101E700045040E949035E8A5E0931D040E9490352A
:101E8000E9A5E0931E040E949035EAA5E0931F04A3
:101E90000E949035ECA1E09316040E949035EDA1CC
:101EA000E09317040E949035EEA1E09318040E947D
:101EB0009035EB89FC89E0934804F09349040E9433
:101EC0009035E0913303E09319040E949035E0913E
:101ED0003503E0931A040E949035E0913403E093B7
:101EE0001B040E949035EB85E0931C040E94903502
:101EF000EF89F88DE0934A04F0934B040E949035EB
:101F0000ED85FE85E0935A04F0935B040E949035C2
:101F10000E9494350E9490350E94DA35E0934E0479
:101F2000F0934F040E949035E0917B03F0917C0385
:101F3000E0935204F09353040E949035E0E023FCB8
:101F4000E1E0E09320040E9490350E947C32E0930F
:101F50005004F09351040E949035E0910603E09301
:101F600021040E949035E0910803E09322040E942E
:101F70009035E0910903E09323040E949035E091AD
:101F80000A03E09324040E949035E0910B03E09350
:101F900025040E949035E0910C03E09326040E94F2
:101FA00090350E94A8310E945932A4E5B4E00E9405
:101FB0004A310E949035E0912A03E09327040E9461
:101FC0009035E0912B03E09328040E949035E09136
:101FD0002C03E09329040E949035E0912D03E093B7
:101FE0002A040E949035E0912E03E0932B040E9476
:101FF0009035E0912F03E0932C040E949035E091FE
:102000003003E0932D040E949035E0913103E0937A
:102010002E040E9490350E949F35E0910E03E093BC
:102020002F040E949035E0E036FCE1E0E0933004BC
:102030000E949035E0911003E09333040E949035A4
:10204000EF8DE09334040E949035EF85F889E0939A
:102050005804F09359040E949035E0914103E093B5
:1020600035040E949035E0914203E09336040E94CB
:102070009035E0914303E09337040E949035E0915E
:102080001E03E09338040E949035E0912003E09312
:1020900039040E949035E0912203E0933A040E94B3
:1020A0009035E0912303E0933B040E949035E0914A
:1020B0001503E0933C040E9490350E9446320E9432
:1020C0009035E0914A03E0933D040E949035E09101
:1020D0004B03E0933E040E949035E0914C03E09363
:1020E0003F040E949035E0914E03E0934004E1E00C
:1020F0004E2E0E94CE35A0E0F1FCA1E00E94FC34FF
:10210000AE81E4E60E94063E0E94813551F068945B
:10211000F1F8EE81EF5FEE83AE81A43611F4E0E0DA
:10212000EE83EAE0E61510F4E894F0F80E94A53397
:10213000A0E0F0FCA1E00E94FC34AE81E0E00E944F
:10214000013E0E94813551F06894F0F8EE81E15033
:10215000EE83AE81AF3F11F4E3E6EE830E94953348
:102160000E94DF35C1F00E94E535A9F4A0913A0341
:10217000A43119F4E7E0E0933A03E0E0E0933B0395
:10218000E894F3F8A0913A03A33028F0E0913A03E1
:10219000E150E0933A03AB2DEAE00E94153E0E2E8B
:1021A0000E94DF35C1F00E94E535A9F4A0913A0301
:1021B000A43119F4E7E0E0933A03E0E0E0933B0355
:1021C000E894F2F8A0913A03A33028F0E0913A03A2
:1021D000E150E0933A03AB2D0E94AA35AA2DEAE024
:1021E0000E941A3EE02131F0E0E0E0933B03E4E19D
:1021F000E0933A03EAE0EA1510F4E894F3F80E9459
:1022000095330E949B330E94F73DE02109F424C3DB
:102210006894F3F8AE81A13049F4A0911703A1307E
:1022200028F4E0911703EF5FE0931703AE81A2302B
:1022300049F4A0911803AF3528F4E0911803EB5F3F
:10224000E0931803AE81A33049F4A0911903A63995
:1022500028F4E0911903EF5F0E94F035AE81A430BD
:1022600049F4A0911B03A83228F4E0911B03EF5F0F
:10227000E0931B03AE81A53031F4ACA5A43618F46D
:10228000ECA5EF5FECA7AE81A63031F4ADA5A43686
:1022900018F4EDA5EF5FEDA7AE81A73031F4AEA540
:1022A000A43618F4EEA5EF5FEEA7AE81A83049F48E
:1022B000A0911C03AF3F28F4E0911C03EF5FE09373
:1022C0001C03AE81A93049F4A0914103AF3F28F42B
:1022D000E0914103EF5FE0934103AE81AA3049F4FE
:1022E000A0914203AF3F28F4E0914203EF5FE093F7
:1022F0004203AE81AB3049F4A0914303AF3F28F4D1
:10230000E0914303EF5FE0934303AE81AC3049F4C7
:10231000A0910E03A03328F4E0910E03E45FE09354
:102320000E03AE81AD3069F4A0915903B0915A0308
:10233000A43CE9E0BE0728F40E942C3331960E94A9
:10234000BD32AE81AE3031F4A8A5A43618F4E8A5AC
:10235000EB5FE8A7AE81AF3031F4A9A5A43618F43D
:10236000E9A5EB5FE9A7AE81A03131F4AAA5A436B7
:1023700018F4EAA5EB5FEAA7AE81A13131F4ACA174
:10238000A83C18F4ECA1EB5FECA3AE81A23131F4D0
:10239000ADA1A83C18F4EDA1EB5FEDA3AE81A33194
:1023A00031F4AEA1A83C18F4EEA1EB5FEEA3AE8130
:1023B000A43169F4A0916903B0916A03A835E2E001
:1023C000BE0728F40E947C327E960E94D432AE81F1
:1023D000A53189F4A0910E03EAE0EA9FF001EA5BDF
:1023E000FF4FAB89BC89AE17BF0728F4EB89FC8986
:1023F0003196EB8BFC8BAE81A63149F4A09133036F
:10240000A13028F4E0913303EF5FE0933303AE8112
:10241000A73149F4A0913503A23328F4E0913503A4
:10242000EF5FE0933503AE81A83149F4A091340306
:10243000A13028F4E0913403EF5FE0933403AE81E0
:10244000A931E1F4AB85BC85E9E1F0E00E940336F7
:102450000E946B3329F0EB85FC853196EB87FC8776
:10246000AB85BC85E2E3F0E00E9403360E9478343D
:1024700029F0EB85FC853196EB87FC87AE81AA318C
:1024800059F40E940A36A03BE4E0BE0728F40E94FB
:10249000DA3531960E940F36AE81AB3191F40E944D
:1024A000BA31A73EE3E0BE07E0E08E07E0E09E071A
:1024B00040F40E948231EF5FFF4F6F4F7F4F0E94C9
:1024C000CB32AE81AC3161F4A0E023FCA1E0A130BD
:1024D00038F4E0E023FCE1E0EF5F0E946C3F23F87A
:1024E000AE81AD3169F40E943231AE3DE3E0BE070A
:1024F00038F40E9413313A96E0936103F09362033B
:10250000AE81AE3169F40E943C31A835E2E0BE07ED
:1025100038F40E941F313A96E0936D03F0936E03F6
:10252000AE81AF3149F4A0910603AA3028F4E091BE
:102530000603EF5FE0930603AE81A03249F4A09159
:102540000803AC3028F4E0910803EF5FE093080340
:10255000AE81A13249F4A0910903AC3028F4E09196
:102560000903EF5FE0930903AE81A23249F4A09121
:102570000A03AC3028F4E0910A03EF5FE0930A030A
:10258000AE81A33249F4A0910B03AC3028F4E09162
:102590000B03EF5FE0930B03AE81A43249F4A091EB
:1025A0000C03AC3028F4E0910C03EF5FE0930C03D4
:1025B000AE81A53249F4A0912A03A13028F4E0911C
:1025C0002A03EF5FE0932A03AE81A63249F4A0917B
:1025D0002B03A13028F4E0912B03EF5FE0932B0352
:1025E000AE81A73249F4A0912C03A23028F4E091E7
:1025F0002C03EF5FE0932C03AE81A83249F4A09145
:102600002D03A13028F4E0912D03EF5FE0932D031B
:10261000AE81A93249F4A0912E03A23028F4E091B2
:102620002E03EF5FE0932E03AE81AA3249F4A0910E
:102630002F03A33028F4E0912F03EF5FE0932F03E3
:10264000AE81AB3249F4A0913003A13028F4E0917F
:102650003003EF5FE0933003AE81AC3249F4A091D8
:102660003103A13028F4E0913103EF5FE0933103AF
:10267000AE81AD3291F40E945032AF39E6E8BE0728
:10268000E1E08E07E0E09E0740F40E943432E65F0E
:10269000FF4F6F4F7F4F0E943D32AE81AE3259F4F3
:1026A0000E942836A031E7E2BE0728F40E949E313E
:1026B0003A960E94A331AE81AF3261F4A0E036FCBD
:1026C000A1E0A13038F4E0E036FCE1E0EF5F0E94E9
:1026D0006C3F36F8AE81A03349F4A0911003A130CD
:1026E00028F4E0911003EF5FE0931003AE81A13373
:1026F00031F4AF8DA33018F4EF8DEF5FEF8FAE8123
:10270000A23359F4AF85B889A632E2E0BE0728F4B7
:10271000EF85F8893196EF87F88BAE81A33349F4C2
:10272000A0911503A43628F4E0911503EF5FE09320
:102730001503AE81A43341F40E942D36A23820F453
:102740000E943436EF5FEC93AE81A53349F4A0913B
:102750004E03A13028F4E0914E03EF5FE0934E0367
:10276000AE81AC3549F4A0910503AA3F28F4E0916D
:102770000503EB5FE0930503AE81AD3531F4AFA502
:10278000A93018F4EFA5EF5FEFA7AE81AE3549F49D
:10279000A0914903A93028F4E0914903EF5FE09349
:1027A0004903AE81AF3559F4AF89B88DA83BEBE052
:1027B000BE0728F4EF89F88D3196EF8BF88FAE8144
:1027C000A03659F4AD85BE85A83EE3E0BE0728F4E7
:1027D000ED85FE853A96ED87FE87AE81A13649F4F8
:1027E000A0912603AC3328F4E0912603EF5FE09339
:1027F0002603AE81A23691F40E94B835A081AA3F8B
:1028000021F40E943B36EB5FEC930E94B835A08127
:10281000AA3F20F40E943B36E65FEC930E944236CA
:102820000E94373EE02149F0A0911D03AA3F28F401
:10283000E0911D03E65FE0931D030E9442360E9473
:10284000433EE02149F0A0911E03AA3F28F4E09105
:102850001E03E65FE0931E03EAE0EB1510F4E89434
:10286000F2F8AB2DEAE00E94153E0E2EA0E0F2FC3D
:10287000A1E00E94FC340E94DF3509F40EC3689485
:10288000F2F8AE81A13049F4A0911703A13028F0ED
:10289000E0911703E150E0931703AE81A23049F4B1
:1028A000A0911803AB3028F0E0911803E550E093B5
:1028B0001803AE81A33049F4A0911903AD3328F079
:1028C000E0911903E1500E94F035AE81A43049F443
:1028D000A0911B03A53128F0E0911B03E150E09388
:1028E0001B03AE81A53031F4ACA5A13018F0ECA5E6
:1028F000E150ECA7AE81A63031F4ADA5A13018F0BF
:10290000EDA5E150EDA7AE81A73031F4AEA5A13021
:1029100018F0EEA5E150EEA7AE81A83049F4A091E1
:102920001C03A13028F0E0911C03E150E0931C034C
:10293000AE81A93049F4A0914103A13028F0E09183
:102940004103E150E0934103AE81AA3049F4A091E4
:102950004203A13028F0E0914203E150E0934203AA
:10296000AE81AB3049F4A0914303A13028F0E0914F
:102970004303E150E0934303AE81AC3049F4A091AE
:102980000E03A93128F0E0910E03EC50E0930E0302
:10299000AE81AD3069F4A0915903B0915A03A538C6
:1029A000E3E0BE0728F00E942C3331970E94BD322D
:1029B000AE81AE3031F4A8A5A63018F0E8A5E550F8
:1029C000E8A7AE81AF3031F4A9A5A63018F0E9A58B
:1029D000E550E9A7AE81A03131F4AAA5A63018F0E0
:1029E000EAA5E550EAA7AE81A13131F4ACA1A1304E
:1029F00018F0ECA1E550ECA3AE81A23131F4ADA109
:102A0000A13018F0EDA1E550EDA3AE81A33131F472
:102A1000AEA1A13018F0EEA1E550EEA3AE81A43135
:102A200061F4A0916903B0916A030E94583F28F4B1
:102A30000E947C327E970E94D432AE81A53189F407
:102A4000A0910E03EAE0EA9FF001E654F040AB8962
:102A5000BC89EA17FB0728F4EB89FC893197EB8BDB
:102A6000FC8BAE81A63149F4A0913303A13028F04C
:102A7000E0913303E150E0933303AE81A73149F491
:102A8000A0913503A23028F0E0913503E150E093A6
:102A90003503AE81A83149F4A0913403A13028F068
:102AA000E0913403E150E0933403AE81A93149F45D
:102AB000AB85BC85129728F0EB85FC853197EB87B9
:102AC000FC87AE81AA3159F40E940A36A73DE1E0A5
:102AD000BE0728F00E94DA3531970E940F36AE818A
:102AE000AB3191F40E94BA31AB30E0E0BE07E0E0D8
:102AF0008E07E0E09E0740F00E948231E150F040F6
:102B0000604070400E94CB32AE81AC3159F4A0E0FD
:102B100023FCA1E0A13030F0A0E023FCA1E00E9462
:102B2000483623F8AE81AD3161F40E9432310E9403
:102B3000583F38F40E9413313197E0936103F093CA
:102B40006203AE81AE3161F40E943C310E94583F75
:102B500038F40E941F313197E0936D03F0936E03B8
:102B6000AE81AF3149F4A0910603A23028F0E09184
:102B70000603E150E0930603AE81A03249F4A09130
:102B80000803A23028F0E0910803E150E093080325
:102B9000AE81A13249F4A0910903A13028F0E0915F
:102BA0000903E150E0930903AE81A23249F4A091F8
:102BB0000A03A13028F0E0910A03E150E0930A03F0
:102BC000AE81A33249F4A0910B03A13028F0E0912B
:102BD0000B03E150E0930B03AE81A43249F4A091C2
:102BE0000C03A13028F0E0910C03E150E0930C03BA
:102BF000AE81A53249F4A0912A03A13028F0E091DA
:102C00002A03E150E0932A03AE81A63249F4A09151
:102C10002B03A13028F0E0912B03E150E0932B032C
:102C2000AE81A73249F4A0912C03A13028F0E091A5
:102C30002C03E150E0932C03AE81A83249F4A0911B
:102C40002D03A13028F0E0912D03E150E0932D03F6
:102C5000AE81A93249F4A0912E03A13028F0E09171
:102C60002E03E150E0932E03AE81AA3249F4A091E5
:102C70002F03A13028F0E0912F03E150E0932F03C0
:102C8000AE81AB3249F4A0913003A13028F0E0913D
:102C90003003E150E0933003AE81AC3249F4A091AF
:102CA0003103A13028F0E0913103E150E09331038A
:102CB000AE81AD3269F40E9450320E945C3F40F414
:102CC0000E943432E150F040604070400E943D323A
:102CD000AE81AE3251F40E9428360E94583F28F44B
:102CE0000E949E3131970E94A331AE81AF3259F4D8
:102CF000A0E036FCA1E0A13030F0A0E036FCA1E07D
:102D00000E94483636F8AE81A03349F4A0911003F2
:102D1000A13028F0E0911003E150E0931003AE8160
:102D2000A13331F4AF8DA13018F0EF8DE150EF8F6A
:102D3000AE81A23359F4AF85B889A93CE0E0BE0763
:102D400028F0EF85F8893197EF87F88BAE81A333B0
:102D500049F4A0911503A23028F0E0911503E15049
:102D6000E0931503AE81A43341F40E942D36A531C2
:102D700020F00E943436E150EC93AE81A53349F443
:102D8000A0914E03A13028F0E0914E03E150E09372
:102D90004E03AE81AC3549F4A0910503A13028F073
:102DA000E0910503E550E0930503AE81AD3531F4C4
:102DB000AFA5A13018F0EFA5E150EFA7AE81AE3579
:102DC00049F4A0914903A13028F0E0914903E15072
:102DD000E0934903AE81AF3559F4AF89B88DA13D79
:102DE000E7E0BE0728F0EF89F88D3197EF8BF88F79
:102DF000AE81A03659F4AD85BE85A536E0E0BE07AC
:102E000028F0ED85FE853A97ED87FE87AE81A136E5
:102E100049F4A0912603A13028F0E0912603E15067
:102E2000E0932603AE81A236D1F40E94B835BF01EB
:102E3000A0810E945D32FB01A081EFEF0E94153E50
:102E4000E02121F00E943B36EA50EC930E94B83515
:102E5000A081AF3F21F40E943B36E550EC930E94E5
:102E600042360E94373EE02149F0A0911D03A13077
:102E700028F0E0911D03EA50E0931D030E944236C2
:102E80000E94433EE02149F0A0911E03A13028F0AA
:102E9000E0911E03EA50E0931E0323FC6FC00E94E2
:102EA0004F36AF8D0E94B433AF8DE3E00E94F73D03
:102EB000E02941F00E944F360E941F350E94C23225
:102EC0000E9459360E941F35E0E0F0E06EEF72E498
:102ED0000E948B3D09F008F40AC00E946236A0E00F
:102EE000B0E080E893E40E94A13C0E945936E09152
:102EF0004803F0E0E0939F03F093A0030E946B3639
:102F0000A038E0E0BE0754F0E0919F03F091A003E9
:102F1000E050F140E0939F03F093A003AF8DA33006
:102F200009F10E941F350E945C3F3CF40E947036FC
:102F30000E94A83C0E94763614C0A091F603AA23F2
:102F40003AF40E9470360E94A13C0E94763609C075
:102F5000E0E0E093E303E093E403E093E503E09330
:102F6000E60304C00E9462360E9476360E947F36D5
:102F7000ADE8B3E00E94D2310E94813623FE45C005
:102F8000EF81F8850E943C350E943B3F0E94363F0E
:102F9000E0E0F0E060E874E40E94463DA0E0B0E4C8
:102FA0008CE995E40E94F83CDF01CB01EF89F88DB4
:102FB0000E9428350E947431DF01CB01E3E3F3E383
:102FC00065E872E40E94463D0E945936A0910F03C5
:102FD000A13048F4E0E0E093F303E093F403E093DE
:102FE000F503E093F6030E9462360E947636E09184
:102FF0000603A0910703AE1740F00E947F36ADE8AC
:10300000B3E00E94D2310E948136A0E0F0FCA1E042
:10301000E0E00E94F73D0E2EE0910603A091070329
:103020000E94103EE02109F446C0E0912D03E030FB
:10303000F1F4A985BA85E0E0F4E00E948536A3E9C1
:10304000B3E00E94D231E0919B03F0919C030E9477
:103050009736A5E9B3E00E94D231E0919D03F0914B
:103060009E030E949736A7E9B3E00E94D231A09157
:103070002D03A130E9F4AF81B885E2E0F0E00E94D1
:10308000B43E3597E0939303F0939403E0919B0350
:10309000F0919C033597E0939503F0939603E091AC
:1030A0009D03F0919E033597E0939703F093980367
:1030B000E0E0E0930703F0916F03E0E0DF01E091CF
:1030C0003903F0E0EA0FFB1FA3ECB3E00E941831D4
:1030D0000E949E36A0E0B0E080E192E40E94463D6E
:1030E0007F936F93FF93EF930E940A360E94A73657
:1030F000AF91BF918F919F910E9428350E94F83C1B
:10310000E093C303F093C4036093C5037093C603B5
:103110000E94AC36E0E0F0E060E87FE30E94B13D61
:103120000E2E0E94AC36E0E0F0E068EC72E40E9403
:10313000AB3DE02109F10E949E36A0E0B0E080E0C6
:103140009FE30E94A83CABEAB3E00E94373C0E9498
:10315000313F0E949E36E093C703F093C80360930B
:10316000C9037093CA030E94AC360E945932ABE582
:10317000B3E00E944A3115C0E0E0E093AB03E09376
:10318000AC03E093AD03E093AE03E093C703E09399
:10319000C803E093C903E093CA03E0935B03E093A1
:1031A0005C030E94DE310E946A310E94B13DEF93C0
:1031B0000E94B5360E94B13DAF91EA23C1F10E9451
:1031C0006131E0E0F0E068EC72E40E94463D0E946C
:1031D000BA310E94403F0E9474310E94B736A091DC
:1031E000BF03B091C0038091C1039091C203E0E09E
:1031F000F0E064E172E40E94F83CDF01CB010E9440
:10320000F5310E94463DA0E0B0E080E291E40E94EA
:10321000F83C0E94B736E091BF03F091C003609183
:10322000C1037091C203DE0114960E94D2310E9444
:10323000A533A0912403EDEF0E94153E0E220E94BB
:103240005934E02129F0E0912403EF5FE093240357
:10325000A62D0E94AA35A0912403EFEF0E94153EEF
:103260000E220E945934E02129F0E894F0F8E0E0C1
:10327000E0932403A0912403EEE10E94F73D0E2E7B
:103280000E945934E02119F0E1E0E0932703E09136
:103290002603E03019F4E0E0E09327030E94C036F3
:1032A0000E948835A0912703E0E00E941A3EE021A9
:1032B00019F0E1E0E0932703A0912703AC3321F458
:1032C000EFEFF0E0E98FFA8FA0910503A13028F02D
:1032D000E0910503F0E00E948033A09131030E9449
:1032E000B4330E947735E02159F1EE8DEF5FEE8F18
:1032F000F0E03196BF01A98DBA8D0E94A736E6177E
:10330000F70790F40E94C5360E94513E0E2E0E948F
:10331000D236E4EAF1E060E070E00E94493EE02944
:1033200019F0E0E0E98FEA8FA98DBA8D0E94A736E7
:10333000AE8DB0E0EA17FB0710F4E0E0EE8F02C0BC
:10334000E0E0EE8F0E9477350E2E0E94C5360E9477
:10335000613E0E22AF85B889E4EAF1E00E94253E85
:10336000E02151F0A98DBA8DA639E0E0BE0720F426
:10337000E6E9F0E0E98FFA8FEF8DE03009F086C0E2
:10338000442041F5E0911403E03041F4E12FF0E0F6
:1033900034960E945233EA0FFB1F03C00E94C133D0
:1033A0003F96A98DBA8D0E94DB36AEE30E94F430C1
:1033B000A4E00E94F430E0911403E03011F4A12F56
:1033C00001C0ABE00E94F430A0E00E94E236A98D7B
:1033D0000E94E836E1E0E41509F058C04424A091C9
:1033E0001903B0E0E2E0F0E00E94B43EE0931A037B
:1033F000F0E0BC96DF01E0911603F0E0AE0FBF1FD6
:10340000E0911703F0E0AE0FBF1FE09118030E9498
:10341000F336AE0FBF1FECA5F0E0AE0FBF1FEDA55A
:10342000F0E0AE0FBF1FEEA5F0E0AE0FBF1FE091C2
:103430001C030E94FA36F0E0AE0FBF1FE091430379
:10344000F0E00E94DB36AEE30E94F430ACE20E9472
:103450000537A09118030E94F430A0911A030E942E
:103460000F37ACA50E94F430ADA50E94F430AEA594
:103470000E941537A09141030E94F430A0914203AD
:103480000E94F430A09143030E94E836AF8DA13032
:1034900009F06DC0A98DBA8DA93CE0E0BE0720F00F
:1034A000E8ECF0E0E98FFA8FE0911B03AFE2AE2782
:1034B000E1E0AE27E6E3EA277E2FA98DBA8DE5E0AD
:1034C0000E94913EE7277E2F8F2F0E945233E5E026
:1034D0000E94913EA72FB82FAE27BF27E1E0F0E072
:1034E000AE27BF27E6E3F0E0AE27BF27E091180341
:1034F000F0E0AE27BF27E12FF0E0AE27BF27E1E0E5
:10350000F0E0EA27FB27E0935D03F0935E03AFE270
:103510000E94F430A1E00E94F430A0E00E940F3736
:103520000E941B37A98DBA8DE5E00E94913EE98F7C
:10353000FA8FAA8D0E94F430A98D0E94F4300E9467
:103540005233E5E00E94913E0E948033E0915003A7
:10355000AE2F0E94E2360E941B37A0E00E94F4309A
:10356000A09118030E94F430A12F0E942137AF8D43
:10357000A33009F092C0442009F045C0E091140343
:10358000E03051F4E12FF0E03596DF01E0914403A3
:10359000F0E0AE0FBF1F05C0E0914403F0E070966D
:1035A000DF01E0914503F0E0AE0FBF1FE09146035D
:1035B000F0E0EA0FFB1F0E945233EA0FFB1FA98DB8
:1035C000BA8D0E94DB36AEE60E94F430A5E00E9480
:1035D000F430E0911403E03011F4A12F01C0ABE00E
:1035E0000E94F430A09144030E94F430A09145035E
:1035F0000E94F430A09146030E94E236A98D0E94F9
:1036000027370E942137E1E0E41509F046C0442441
:10361000E0911603F0E0BD96DF01E09117030E94F0
:10362000FA360E94F336AE0FBF1FD296E0911C030C
:10363000F0E0AE0FBF1FE0911503F0E0EA0FFB1FB3
:103640007E2F8F2FAB85BC85EAE00E94913EE70F6D
:10365000F81FE0935D03F0935E03AEE60E94F43042
:10366000ADE20E940537A09142030E94F430A09180
:1036700041030E940F37A2E30E9427370E941537AB
:10368000EB85AAE0EA9FF001AE2F0E94F430A091F2
:1036900015030E9427370E942137E09141040E94C0
:1036A0006232FF27662777270E94623F24F4E09169
:1036B000AB03E0934104E09142040E941F35FF27D1
:1036C000662777270E946E3C0E948B3D09F008F424
:1036D00007C00E946236A2E4B4E00E94353CEC933D
:1036E000E09143040E946B36F0E0EA17FB0724F4F4
:1036F000E0919F03E0934304E0915C04F0915D044A
:103700000E942E37662777270E94593E0E2E0E9470
:103710002E37E8ECF0E060E070E00E94613EE021CE
:1037200041F0E091B303F091B403E0935C04F093B3
:103730005D04E0915E04F0915F040E942E376627DD
:1037400077270E94623F44F4E091B303F091B40301
:10375000E0935E04F0935F04E0916204F0916304EF
:10376000A0919303B0919403EA17FB0740F4E09112
:103770009303F0919403E0936204F0936304A091A7
:103780009503B0919603E0916404F09165040E9462
:10379000433E0E948A340E946234E02141F0E0916D
:1037A0009503F0919603E0936404F0936504A0916F
:1037B0009703B0919803E0916604F09167040E942A
:1037C000433E0E948A340E946234E02141F0E0913D
:1037D0009703F0919803E0936604F0936704A09137
:1037E0006804B09169040E94A535EA1BFB0BE4361E
:1037F000A0E0FA0730F00E94A535E0936804F0934A
:103800006904E091B303F091B4036091B503709142
:10381000B6030E941F350E946E3C0E94F83CA1EA4C
:10382000B3E00E94D2310E9437370E943C37E093C8
:10383000A103F093A203E0916004F09161040E945F
:103840003737EA17FB0740F4E091A103F091A20398
:10385000E0936004F0936104033608F0DAC70E9435
:10386000D4350081A0913703A13048F420FC07C073
:10387000A0E0F799A1E0EA2FE295E07F19C0A0E06F
:10388000F799A1E0EA2FE295E07F0E2EA0E0F399F0
:10389000A1E0EA2FEE0FEE0F0E0EA0E0F499A1E0EA
:1038A000EA2FEE0FA02DAE0FE0E0F599E1E0EA0F70
:1038B000E8AB0E941F35EDECFCEC6CEC7DEB0E945C
:1038C0008B3D18F4E8A9E05AE8ABEAE00E944137E2
:1038D000EAE0DE01AC5BBF4FEC930E9446370E94EA
:1038E0004C37EAE00E945137EAE00E945637EAE09E
:1038F0000E945B370E946037E89435F8A0E031FC05
:10390000A1E00E94B433A0E032FCA1E0E1E00E941B
:10391000F73D0E2AA0E034FCA1E0E1E00E94F73D73
:10392000E02911F020FA01C0E894F5F8E0912F03A6
:10393000E03021F40E9482370E949237A0912F0339
:10394000A13081F4A0E022FCA1E0EA2FEE0FE75FB6
:103950000E2EA0E022FCA1E0EA2FEE0FEE0FE00D0C
:103960000E94A137A0912F03A23099F40E948237C0
:10397000A0E022FCA1E0EA2F0E94B1370E0EA0E0E9
:1039800022FCA1E0EA2FE295E07FEE0F0E0E0E94EE
:103990009237A0912F03A33031F4E0E022FCE1E064
:1039A000E85F0E94A137A0910E03A83109F041C041
:1039B0000E94B637A23DE0E0BE07E0E08E07E0E0FF
:1039C0009E071CF0E1E0E09301030E942E37A83F20
:1039D000E0E0BE07E0E08E07E0E09E071CF0E3E0D9
:1039E000E09301030E942E37AF3FE0E0BE07E0E026
:1039F0008E07E0E09E071CF0E7E0E09301030E94E1
:103A00002E37A430E1E0BE07E0E08E07E0E09E073D
:103A10001CF0EFE0E09301030E942E37AE30E1E0AE
:103A2000BE07E0E08E07E0E09E071CF0EFE1E093C8
:103A30000103A0910E03A43209F041C00E94B637E1
:103A4000A633E1E0BE07E0E08E07E0E09E071CF051
:103A5000E1E0E09301030E942E37AA34E1E0BE07C3
:103A6000E0E08E07E0E09E071CF0E3E0E093010356
:103A70000E942E37AE35E1E0BE07E0E08E07E0E0C1
:103A80009E071CF0E7E0E09301030E942E37A83662
:103A9000E1E0BE07E0E08E07E0E09E071CF0EFE00B
:103AA000E09301030E942E37AC37E1E0BE07E0E06F
:103AB0008E07E0E09E071CF0EFE1E0930103A09188
:103AC0000E03A03309F041C00E94B637A638E1E0EA
:103AD000BE07E0E08E07E0E09E071CF0E1E0E09327
:103AE00001030E942E37AC3CE1E0BE07E0E08E0708
:103AF000E0E09E071CF0E3E0E09301030E942E3714
:103B0000A63DE1E0BE07E0E08E07E0E09E071CF086
:103B1000E7E0E09301030E942E37A03EE1E0BE07FC
:103B2000E0E08E07E0E09E071CF0EFE0E093010389
:103B30000E942E37AF3EE1E0BE07E0E08E07E0E0F6
:103B40009E071CF0EFE1E0930103A0911403A13064
:103B500081F4A0E020FCA1E0EA2F0E94B1370E2EF4
:103B6000A0E020FCA1E0EA2FE295E07FEE0FE00D5F
:103B70004E0FA0910203A431F0F40E9462320E9421
:103B8000BC376CF0FE01EE5BFF4F3396FF93EF9373
:103B90000E94C4370E94CA37AF91BF91EC930E9434
:103BA000D537FF93EF930E94C4370E94F83EAF9140
:103BB000BF91EC930DC020FE05C0E0E40E94DA370F
:103BC000E0E402C00E944637DE01AA5BBF4FEC93DF
:103BD000AD8DA13090F0ED8DE150ED8FE8E70E94C2
:103BE000DA37E0911403E03029F4FE01EE5BFF4F79
:103BF000148303C0E0E50E944C37AC8DA13058F02F
:103C0000EC8DE150EC8FE8E30E94DA370E94D53763
:103C1000A0913203A083AB8DA13048F0EB8DE15031
:103C2000EB8FE9E30E94DA37E0E50E944C37E09140
:103C30001103E03019F54058A0918E03AA2392F4A5
:103C4000E0E40E944137A0918D03B0918E03AD391D
:103C5000EFEFBE0714F4689435F80E94DF370E9436
:103C6000E73702C0E89435F80E94EC371A9724F041
:103C70000E94F1370E94F8370E940038A09111038A
:103C8000A13009F045C0E8A9E85FE8AB0E940D3813
:103C9000FF2392F4E0E40E9441370E940D38E73F91
:103CA000AFEFFA0714F4689401C0E89435F80E9465
:103CB0000D380E94C13D04C0E89435F80E940D38CB
:103CC000E0938F03F09390030E94EC371A9724F04F
:103CD0000E94F1370E94F8370E9400380E940D3888
:103CE000BF01DF01E3E6F0E00E94313E0E2EDB0172
:103CF000EDE9FFEF0E942B3EE02951F0E89435F802
:103D0000E0E40E944137E0E4DE01AC5BBF4FEC939E
:103D10000E941938FF93EF930E942E370E941E389D
:103D20000E94CA37AF91BF910E9423383696FF9305
:103D3000EF930E9428380E94CA37AF91BF910E942A
:103D400023383796FF93EF930E9428380E94F83E5D
:103D5000AF91BF91EC930E942E37A639E0E0BE07E9
:103D6000E0E08E07E0E09E0764F4E0E40E94513753
:103D7000E0E40E945637E0E40E945B37E0E0E09325
:103D80000103013009F05BC00E942E380E943638D2
:103D9000A83EE3E0BE07B8F0505E0E943B380E94A8
:103DA00041380E9423383E96BF010E9436380E9457
:103DB0004C380E9423383F96BF010E9436380E943B
:103DC000A736DF011BC050560E943638A436E0E00B
:103DD000BE0728F00E943B380E944C38EC930E94AA
:103DE0005738BF010E9436380E94A7360E945C38BF
:103DF0000E9423383F96BF010E943638EAE0F0E087
:103E00000E946338A0910003AA3010F00E94683825
:103E10000E946E38A09100030E9474380E942338DB
:103E20003A96BF01AC2DB0E00E943C370E94F837B3
:103E30000E947B38BF01AC2D0E947438EC93023095
:103E400009F06DC0505C0E945032A03AE6E8BE070F
:103E5000E1E08E07E0E09E0778F00E948038FF9353
:103E6000EF930E945032E0EAF6E861E070E00E94D1
:103E70008538AF91BF91EC930E9450320E949038E8
:103E800078F00E947B38FF93EF930E945032E0E17C
:103E9000F7E260E070E00E948538AF91BF91EC934B
:103EA0000E9450320E94983868F00E94A038FF9318
:103EB000EF930E9450320E9454340E948538AF9193
:103EC000BF91EC930E9450320E94A53868F00E9486
:103ED000AD38FF93EF930E9450320E941E380E942B
:103EE0008538AF91BF91EC930E9450320E94BC374D
:103EF00058F00E945738FF93EF930E94B2380E9407
:103F00008538AF91BF91EC930E94B838FF93EF933F
:103F10000E94B2380E94F43EAF91BF91EC930330FF
:103F200009F08FC0E7E70E94BD38A091BA03AA2329
:103F300092F4E091B703F091B8036091B9037091E6
:103F4000BA030E94C53DE093B703F093B8036093B2
:103F5000B9037093BA030E94B5360E947431772377
:103F600012F40E94C7380E94B5360E9474310E9434
:103F7000CD3810F40E94D6380E94B5360E947431B4
:103F80000E94DC3810F40E94E5380E94B5360E9489
:103F900074310E94EB3810F40E94EE380E94F4381D
:103FA0000E9490387CF00E947B38FF93EF930E9430
:103FB000F438E0E1F7E260E070E00E94CA37AF91C8
:103FC000BF91EC930E94F4380E9498386CF00E94E4
:103FD000A038FF93EF930E94F4380E9454340E945B
:103FE000CA37AF91BF91EC930E94F4380E94A53874
:103FF0006CF00E94AD38FF93EF930E94F4380E945A
:104000001E380E94CA37AF91BF91EC930E94F438DA
:104010000E94BC375CF00E945738FF93EF930E94D8
:10402000FD380E94CA37AF91BF91EC930E94B83817
:10403000FF93EF930E94FD380E94F83EAF91BF912D
:10404000EC93043009F054C05058EEE30E94BD38A0
:10405000A0918A03AA2312F40E9403390E940E3908
:10406000772312F40E94C7380E940E390E94CD387F
:1040700010F40E94D6380E940E390E94DC3810F4E9
:104080000E94E5380E940E390E94EB3810F40E941D
:10409000EE380E941439A031E7E2BE0724F00E94F6
:1040A0007B380E9419390E941439A83EE3E0BE070C
:1040B00024F00E94A0380E9420390E941439A436AE
:1040C000E0E0BE0724F00E94AD380E9427390E942C
:1040D00014391A974CF00E945738BF010E941439C6
:1040E0000E943C370E94F8370E94B8380E942E394F
:1040F000053071F55058EEE30E94BD380E94373903
:10410000A091EA03AA2312F40E94D6380E94DE315D
:10411000E0E0F0E066EC72EC0E948B3D10F40E944F
:10412000E5380E943D39A436E0E0BE0724F00E9445
:10413000AD380E9442390E945738BF010E943D3974
:104140000E943C370E94F8370E94B8380E944939D3
:104150000630A1F55058E0E00E945239E5E00E9497
:104160005739E8E70E945C39AC81BD81A83EE3E0A5
:10417000BE073CF00E94A038BF01AC81BD810E9407
:104180006139AC81BD81A436E0E0BE073CF00E94FD
:10419000AD38BF01AC81BD810E9466390E9457389D
:1041A000BF01AC81BD810E943C370E94F8370E945C
:1041B000B838BF01AC81BD810E946B39073009F06E
:1041C00076C0A98DBA8D0E94583F30F5ECE00E9470
:1041D00052390E947239E436A0E0FA0740F00E949A
:1041E0008038BF01A98DBA8D0E947739EC930E9467
:1041F00072393A9740F00E947B38BF01A98DBA8D81
:104200000E947C39EC930E94A038BF010E94723951
:104210000E945C38EC934BC0E0914203E03029F5FA
:10422000EBE00E9452390E948139E436A0E0FA079F
:1042300040F00E948038BF01A989BA890E9477396D
:10424000EC930E9481393A9740F00E947B38BF017D
:10425000A989BA890E947C39EC930E94A038BF01D9
:104260000E9481390E945C38EC93A0914203A130F6
:10427000F1F4EBE00E945239A989BA89A436E0E052
:10428000BE0740F00E948038BF01A989BA890E9408
:104290004C38EC930E947B38BF01A989BA890E94EF
:1042A000A7360E945C38EC93E7E70E948639083015
:1042B00009F07EC00E942E38A0918503B09186033C
:1042C000A135EBEFBE0734F4E1E5FBEFE0938503A6
:1042D000F0938603A0918503B0918603A03BE4E0B0
:1042E000BE0734F0EFEAF4E0E0938503F093860331
:1042F000A0918603AA234AF40E94E538E091850341
:10430000F09186030E94C13D04C0E0918503F091C5
:104310008603E0938703F0938803A0918703B0910D
:104320008803ECE3F0E00E94B43EE0936303F09373
:1043300064030E948B39ECE30E94913EA0918703B5
:10434000B0918803AE1BBF0BA0936503B0936603C7
:1043500024FE25C00E948B391A9710F00E946838FD
:104360000E946E380E948B39EAE0F0E00E94E33E42
:10437000DB010E9423383A96BF01A0916503B091FA
:1043800066030E94A7360E945C380E9423383B9641
:10439000BF01A0916503B09166030E949039E3E7E5
:1043A0000E949339E8E30E949839E4E50E949D3920
:1043B000093009F056C050580E946838EEE30E9458
:1043C000BD38A0918A03AA2312F40E9403390E94E7
:1043D0000E39772312F40E94C7380E940E390E94CA
:1043E000CD3810F40E94D6380E940E390E94DC3875
:1043F00010F40E94E5380E940E390E94EB3810F448
:104400000E94EE380E941439A031E7E2BE0724F082
:104410000E947B380E9419390E941439A83EE3E0BB
:10442000BE0724F00E94A0380E9420390E9414394F
:10443000A436E0E0BE0724F00E94AD380E94273980
:104440000E9414391A974CF00E945738BF010E94FD
:1044500014390E943C370E94F8370E94B8380E94F5
:104460002E390A30F9F450580E946838EEE30E9461
:10447000BD380E9437390E943D39A436E0E0BE07BE
:1044800024F00E94AD380E9442390E945738BF0183
:104490000E943D390E943C370E94F8370E94B8388C
:1044A0000E9449390B30A1F55054E9E30E94573975
:1044B000E8E30E945C390E942836A83EE3E0BE078C
:1044C00040F00E94A038BF010E9428360E94413867
:1044D000EC930E942836A436E0E0BE0740F00E942C
:1044E000AD38BF010E9428360E944C38EC930E94E0
:1044F0005738BF010E9428360E94A7360E945C38B8
:104500000E9423383F96BF010E9428360E949039AE
:104510000C3009F073C00E946838EEE30E945239F3
:104520000E943737E0E0F0E00E94A239E6EFFFEFAB
:104530000E94313EE02111F00E94C7380E943737B7
:10454000E7EFFFEF0E94A239ECE9FFEF0E94313E56
:10455000E02111F00E94D6380E943737EDE9FFEFD5
:104560000E94A239E8E1FCEF0E94313EE02111F007
:104570000E94E5380E943737A931ECEFBE0714F4EA
:104580000E94EE38A091A203AA2352F4E091A10365
:10459000F091A2030E94C13DE093A103F093A20316
:1045A0000E943737A83EE3E0BE073CF00E94A038E7
:1045B000BF010E9437370E9461390E943737A43605
:1045C000E0E0BE073CF00E94AD38BF010E943737E3
:1045D0000E9466390E9437371A974CF00E9457386C
:1045E000BF010E9437370E943C370E94F8370E9473
:1045F000B838BF010E9437370E946B39AAA10E94C8
:104600005D32A9A1E0E00E941A3EE02909F4AFC0A2
:104610005F77E0913803E170EE0F4E23E0913803AD
:10462000E6950E94A6390E2EE0913803E695E695B0
:10463000E170AE2FE0E0F5FCE1E0EA2BEE0FEE0FCB
:10464000E00D4E0F0E946037A9A10E945D32AAA121
:10465000E0E00E941A3EE02159F1A9A1A13029F41D
:104660000E94AB39ECE00E948639A9A1A23029F45E
:104670000E94AB39EDE00E948639A9A1A33029F44C
:104680000E94AB39EBE00E9486390E94AE3929F0D6
:104690000E94AB39ECE00E9486390E9490330E9460
:1046A000B83929F00E94AB39EBE00E9486392AC064
:1046B000A9A1A13029F40E94BE39ECE00E949D39E5
:1046C000A9A1A23029F40E94BE39EDE00E949D39D3
:1046D000A9A1A33029F40E94BE39EBE00E949D39C4
:1046E0000E94AE3929F00E94BE39ECE00E949D394B
:1046F0000E9490330E94B83929F00E94BE39EBE045
:104700000E949D39AAA1A13029F40E94C239ECE08F
:104710000E949D39AAA1A23029F40E94C239EDE07D
:104720000E949D39AAA1A33029F40E94C239EBE06E
:104730000E949D39AAA1E4E00E94F73D0E94B83989
:1047400029F00E94C239ECE00E949D39AAA1E5E05F
:104750000E94F73D0E94B83929F00E94C239EBE06F
:104760000E949D39E0911103E03009F44058E09136
:104770004A03A0919303B09194030E94C6390E2E70
:10478000A0914A030E94CA3931F0E0E00E94CF397B
:10479000E0E00E94D339A0919503B0919603E09197
:1047A0004B030E94C6390E2EA0914B030E94CA39BA
:1047B00031F0E1E00E94CF39E1E00E94D339A091CD
:1047C0009703B0919803E0914C030E94C6390E2ED6
:1047D000A0914C030E94CA39C1F0E2E00E94CF3997
:1047E000E2E00E945739E0E00E945C39E9E70E946C
:1047F0008639E0E50E949339E0E50E949839E0E0CF
:104800000E949D39E1E0E0933F03F29B02C04B7FA1
:104810004F5F033611F00C94EB2C31E0303140F453
:104820000E94E239EAE0EC93E89435F83F5FF6CF76
:10483000AE81EBE50E94EA39EAE50E94F73DE02906
:1048400011F0E5E3EE83AE81A63311F4ECE5EE83DF
:10485000EE81E03029F4E0911603F0E0ED8BFE8B61
:10486000AE81A13029F4E0911703F0E0ED8BFE8BCF
:10487000AE81A23029F4E0911803F0E0ED8BFE8BBD
:10488000AE81A33029F4E0911903F0E0ED8BFE8BAB
:10489000AE81A43029F4E0911B03F0E0ED8BFE8B98
:1048A000AE81A53021F4ECA5F0E0ED8BFE8BAE815E
:1048B000A63021F4EDA5F0E0ED8BFE8BAE81A730A4
:1048C00021F4EEA5F0E0ED8BFE8BAE81A83029F44B
:1048D000E0911C03F0E0ED8BFE8BAE81A93029F452
:1048E000E0914103F0E0ED8BFE8BAE81AA3029F41C
:1048F000E0914203F0E0ED8BFE8BAE81AB3029F40A
:10490000E0914303F0E0ED8BFE8BAE81AC3029F4F7
:10491000E0910E03F0E0ED8BFE8BAE81AD3021F423
:104920000E942C33ED8BFE8BAE81AE3021F4E8A5D6
:10493000F0E0ED8BFE8BAE81AF3021F4E9A5F0E025
:10494000ED8BFE8BAE81A03121F4EAA5F0E0ED8B7A
:10495000FE8BAE81A13121F4ECA1F0E0ED8BFE8B5A
:10496000AE81A23121F4EDA1F0E0ED8BFE8BAE81A2
:10497000A33121F4EEA1F0E0ED8BFE8BAE81A431EA
:1049800021F40E947C32ED8BFE8BAE81A53121F4A7
:10499000EB89FC89ED8BFE8BAE81A63129F4E09189
:1049A0003303F0E0ED8BFE8BAE81A73129F4E0916B
:1049B0003503F0E0ED8BFE8BAE81A83129F4E09158
:1049C0003403F0E0ED8BFE8BAE81A93121F4EB8551
:1049D000FC85ED8BFE8BAE81AA3121F40E94DA3585
:1049E000ED8BFE8BAE81AB3131F4E0917B03F09126
:1049F0007C03ED8BFE8BAE81AC3131F4E0E023FC27
:104A0000E1E0F0E0ED8BFE8BAE81AD3121F40E9450
:104A10001331ED8BFE8BAE81AE3121F40E941F313C
:104A2000ED8BFE8BAE81AF3129F4E0910603F0E00F
:104A3000ED8BFE8BAE81A03229F4E0910803F0E00B
:104A4000ED8BFE8BAE81A13229F4E0910903F0E0F9
:104A5000ED8BFE8BAE81A23229F4E0910A03F0E0E7
:104A6000ED8BFE8BAE81A33229F4E0910B03F0E0D5
:104A7000ED8BFE8BAE81A43229F4E0910C03F0E0C3
:104A8000ED8BFE8BAE81A53229F4E0912A03F0E094
:104A9000ED8BFE8BAE81A63229F4E0912B03F0E082
:104AA000ED8BFE8BAE81A73229F4E0912C03F0E070
:104AB000ED8BFE8BAE81A83229F4E0912D03F0E05E
:104AC000ED8BFE8BAE81A93229F4E0912E03F0E04C
:104AD000ED8BFE8BAE81AA3229F4E0912F03F0E03A
:104AE000ED8BFE8BAE81AB3229F4E0913003F0E028
:104AF000ED8BFE8BAE81AC3229F4E0913103F0E016
:104B0000ED8BFE8BAE81AD3231F4E0917703F09105
:104B10007803ED8BFE8BAE81AE3221F40E949E3184
:104B2000ED8BFE8BAE81AF3231F4E0E036FCE1E09C
:104B3000F0E0ED8BFE8BAE81A03329F4E091100301
:104B4000F0E0ED8BFE8BAE81A13321F4EF8DF0E030
:104B5000ED8BFE8BAE81A23321F4EF85F889ED8BCE
:104B6000FE8BAE81A33329F4E0911503F0E0ED8BC9
:104B7000FE8BAE81A43349F4E0912C03F0E0E65BB8
:104B8000FC4FE081F0E0ED8BFE8BAE81A53329F484
:104B9000E0914E03F0E0ED8BFE8BAE81AC3529F455
:104BA000E0910503F0E0ED8BFE8BAE81AD3521F495
:104BB000EFA5F0E0ED8BFE8BAE81AE3529F4E091F0
:104BC0004903F0E0ED8BFE8BAE81AF3521F4EF8928
:104BD000F88DED8BFE8BAE81A03621F4ED85FE8540
:104BE000ED8BFE8BAE81A13629F4E0912603F0E037
:104BF000ED8BFE8BAE81A23631F40E94B835E08198
:104C0000F0E0ED8BFE8B0E9442360E94373EE021A1
:104C100029F0E0911D03F0E0ED8BFE8B0E944236FF
:104C20000E94433EE02129F0E0911E03F0E0ED8B6D
:104C3000FE8BAE81E0E00E94EA39E3E00E94EF39AA
:104C4000E1E10E94EF39E2E10E94EF39E3E10E94E5
:104C5000EF39E5E10E94EF39EAE10E94EF39EBE13B
:104C60000E94EF39EDE10E94EF39EEE20E94F73D3C
:104C7000E0291E2E0E94F4390E94253EE0211E2AC2
:104C8000AE81EEE50E94F73D0E2EA0914903E2E0D1
:104C90000E941A3E0E22E5E00E94153EE021E12925
:104CA00011F0F69A01C0F698A0E0F699A1E0EA2F7B
:104CB000E795E0E0E7955E2F40E0E0E0E8ABE093C9
:104CC0000103FE01EE5BFF4F3396BF01AE81B0E002
:104CD000A7FDBFEF0E943C370E94F8370E94D537EE
:104CE000BF01AE81B0E0A7FDBFEF0E946B39AD8977
:104CF000BE89A031E7E2BE0740F00E947B38BF01C9
:104D0000AD89BE890E94FE39EC93AD89BE89A83E6B
:104D1000E3E0BE0740F00E94A038BF01AD89BE8924
:104D20000E944138EC93AD89BE89A436E0E0BE070D
:104D300040F00E94AD38BF01AD89BE890E944C3859
:104D4000EC93AD89BE891A9738F00E9457380E94BB
:104D5000033A0E945C38EC930E94B838BF01AD89D9
:104D6000BE890E949039EE81E03079F4ECE10E9436
:104D7000073AE0E50E945B37EDE60E945739E4E52B
:104D80000E945C39E0E50E948639AE81A13031F4A1
:104D9000EBE50E94073AEDE60E945B37AE81A23058
:104DA00029F40E940A3AE8E30E945B37AE81A330FF
:104DB00049F4EEE50E945137E0E30E945637E7E7F9
:104DC0000E945B37AE81A83011F40E940E3AAE818A
:104DD000AC3031F4EEE30E94143AECE70E945B370A
:104DE000AE81E1E10E94EA39E2E10E94EF39E3E1BC
:104DF0000E94EF39E5E10E94EF39EDE10E94EF39C1
:104E0000EEE20E94F73DE02939F00E9457380E94F7
:104E1000033A0E945C38EC93E7EAE0937A000E9440
:104E20004833E7E2E0937A000E94173AEEE00E94EE
:104E3000EF39E1E10E94F73DE02911F0E1E07E2E3B
:104E4000AE81E6E00E94EA39EFE00E94EF39E2E14C
:104E50000E94F73DE02911F0E2E07E2EAE81E7E00E
:104E60000E94EA39E0E10E94EF390E941A3A11F0FB
:104E7000E3E07E2E0E945233D39708F45DC00E9477
:104E8000C1330E94C633E72D0E94CD3320F0E8ECF9
:104E9000F0E00E948033A0914203A13011F40E94FF
:104EA000DD33E72D0E94E8330E941F3AAC91A13018
:104EB00008F441C00E94263A0E9408340E94673FCD
:104EC0004CF40E941F3A0E942F3A0E94B73D0E9464
:104ED000393A23C00E94423A0E942934EF930E943B
:104EE000423A0E943234AF91EA2379F00E941F3A8D
:104EF0000E942F3A0E94BC3DA093A703B093A80341
:104F00008093A9039093AA0308C00E94423A0E948A
:104F10003B341CF00E94443A0EC0A091A703B0910C
:104F2000A8038091A9039091AA030E9454340E947F
:104F3000DE3E0E94803304C00E9485330E94443AC2
:104F4000AE81AD3029F50E941938FF93EF930E948E
:104F5000D2360E941E380E94CA37AF91BF910E947C
:104F600023383696FF93EF930E94533A0E94CA3734
:104F7000AF91BF910E9423383796FF93EF930E9421
:104F8000533A0E94F83EAF91BF91EC93E0E2E8AB58
:104F9000AE81A53141F4EEE30E945137ECE00E946E
:104FA0005637E0E6E8AB0E94173AEEE00E94EF3990
:104FB000E1E10E94F73DE029B1F00E94593AE4E0B6
:104FC0000E945D3A28F00E9419380E94633AEC93DF
:104FD0000E9452331A9728F00E94663A0E945C3869
:104FE000EC930E946D3AAE81E6E00E94EA39EFE070
:104FF0000E94EF39E2E10E94F73DE029B1F00E9402
:10500000593AE2E00E945D3A28F00E9419380E9465
:10501000633AEC930E9452331A9728F00E94663A42
:105020000E945C38EC930E946D3AAE81E7E00E94EA
:10503000EA39E0E10E94EF390E941A3AB1F00E9489
:10504000593AE1E00E945D3A28F00E9419380E9426
:10505000633AEC930E9452331A9728F00E94663A02
:105060000E945C38EC930E946D3AAE81E5E00E94AC
:10507000743A1E2EAE81E6E00E94743A1E2AAE817A
:10508000E7E00E94743AE12951F1E72DF0E0DE01FA
:105090009B96AE0FBF1FEC91F0E0AB85BC850E94E4
:1050A000693EDF01E4E6F0E00E94A13E0E94803309
:1050B0000E9452331A9750F00E941938BF010E9483
:1050C00052330E94A7360E945C38EC930E947A3AD1
:1050D0000E9452330E949039E7E70E945B37AE810D
:1050E000A431B1F40E9419380E94803A0E944C38D1
:1050F0000E94233836960E94803A0E94A7360E946A
:105100005C380E94233837960E94803A0E9490397A
:10511000AE81A63129F40E940E3AEBE00E9452398A
:10512000AE81A73129F40E940E3AE0E40E94523980
:10513000AE81A83129F40E940E3AECE00E94523967
:10514000AE81A931D1F4A091F603AA2322F40E94E2
:10515000DF370E94E7370E941938BF010E94EC3701
:105160000E943C370E94F8370E947A3A0E94EC373E
:105170000E946B39E7E70E945B37AE81AA31F1F4F8
:105180000E94863AA436E0E0BE0740F00E9419383B
:10519000BF010E94863A0E944C38EC930E947A3AF2
:1051A0000E94863A0E94A7360E945C380E942338EB
:1051B0003796BF010E94863A0E949039AE81AB318A
:1051C00069F4ECE70E94143AE8E70E945B370E941A
:1051D00057380E94033A0E945C38EC93AE81AC31A0
:1051E00049F4E0E30E945137EDE60E945637E4E5CA
:1051F0000E945B37AE81AF3149F4EEE30E94513734
:10520000EDE60E945637E3E70E945B37AE81A53298
:1052100029F40E948B3AE5E00E945B37AE81A6320A
:1052200029F40E948B3AE8E00E945B37AE81A732F6
:1052300029F40E948F3AE3E60E945B37AE81A832E0
:1052400029F40E948F3AE8E70E945B37AE81A932C9
:1052500049F4E7E70E945137E0E40E945637E8E757
:105260000E945B37AE81AB3231F4E9E30E94933A9E
:10527000EEE00E945B37AE81AC3231F4ECE70E9485
:10528000933AEDE60E945B37AE81AD3231F4E0E057
:105290000E94963AE0E00E945B37AE81EDE10E9409
:1052A000EA39EEE10E94F73DE02921F1E3E70E94AF
:1052B0005239E8E30E945739AE81AD3111F4EEE581
:1052C00001C0E8E7DE01A35BBF4FEC930E94993A6F
:1052D0001A9748F00E947A3A0E94993A0E94A7369B
:1052E0000E945C38EC930E949E3ABF010E94993A5A
:1052F0000E9490390E94173AE6E00E94EF39E7E0F9
:105300000E94F73DE02919F0E3E70E945239AE818F
:10531000EEE00E94EA39EFE00E94EF39E0E10E94FE
:10532000F73DE02949F0EDE60E945239E9E70E9495
:105330005739E4E50E945C39AE81E1E10E94EA3927
:10534000E2E10E94EF390E941A3A19F0E8E70E9460
:105350005739AE81EFE10E940B3E0E2EE5E20E942E
:10536000063EE02161F0EDE60E945137E8E50E943B
:1053700056370E949E3ADF01EE81EF51EC93AE81E9
:10538000AE3231F4E9E30E945137E8E30E94563728
:10539000AE81AF3249F4E8E70E945137E5E00E9460
:1053A0005637E7E70E945B37AE81A03331F4E0E384
:1053B0000E94073AE0E50E945B37AE81A133B1F469
:1053C000E3E70E94933AE8E70E945B37A09102036B
:1053D000A43160F0E4E50E945239EDE60E945739AD
:1053E000E0E30E945C39EDE30E948639AE81A2338E
:1053F00041F4EEE30E945137EBE00E945637E0E6BD
:10540000E8AB0E94F4390E941F3EE02111F00E9497
:10541000A33AAE81A33329F40E94A93AE8E30E949B
:105420005B37AE81A43389F4E8E70E945137E8E3A3
:105430000E9456370E949E3AA0912C03A083AD890A
:10544000BE89549711F40E94A33AAE81A53349F462
:10545000E8E30E945137E0E30E945637E4E50E94FA
:105460005B37AE81AC3549F4E7E70E945137E9E399
:105470000E945637E9E30E945B37AE81AD3509F0F3
:1054800086C0AFA5A83008F044C0E7E70E94963A6E
:105490000E949E3AAFA5A083E7EAE0937A000E94BB
:1054A0001333E0935103F0935203E7E2E0937A0061
:1054B0000E94AD3AA83EE3E0BE0740F00E94A0384B
:1054C000BF010E94AD3A0E944138EC930E94AD3A70
:1054D000A436E0E0BE0740F00E94AD38BF010E9454
:1054E000AD3A0E944C38EC930E94AD3A1A9750F0B6
:1054F0000E945738BF010E94AD3A0E94A7360E9411
:105500005C38EC930E94B838BF010E94AD3A0E940B
:105510009039AFA5A830E1F4E6E70E94143AE8E339
:105520000E94B23ADF01E0914703E1700E94233804
:105530003E96DF01E0914703E695E1700E94233833
:105540003F96DF01E0914703E695E695E170EC9325
:10555000AFA5A930E1F40E94A93AE0E30E945B37CD
:105560000E946B361A974CF00E94AD38BF010E9422
:105570006B360E943C370E94F8370E945738BF01B3
:105580000E946B360E946B39E7E70E949D39AE811D
:10559000AE3509F0B8C1E0914903E030D9F40E947A
:1055A0000A3AEBE00E945B37A0914104AA3050F028
:1055B0000E945738BF01A0914104B0E00E943C37DF
:1055C0000E94F8370E94B838BF01A09141040E94A0
:1055D0007438EC93A0914903A130F9F4E0E30E9400
:1055E000B43AEBE00E945B37A0914204AA3050F03D
:1055F0000E94AD38BF01A0914204B0E00E943C3748
:105600000E94F8370E945738BF01A09142040E94BF
:105610007438EC93E7E70E949D39A0914903A230CA
:10562000F9F4E0E30E945137E3E70E94B73AA09112
:105630004304AA3050F00E94AD38BF01A09143044A
:10564000B0E00E943C370E94F8370E945738BF01F3
:10565000A09143040E947438EC93E7E70E949D39BF
:10566000A0914903A330D1F4EEE30E94B43AECE0F8
:105670000E94B23A0E94BA3A0E944C380E942338E3
:105680003E960E94BA3A0E94A7360E945C380E9459
:1056900023383F960E94BA3A0E949039A09149035C
:1056A000A430D1F4EEE30E94B43AEBE00E94B23AA7
:1056B0000E94C03A0E944C380E9423383E960E94B5
:1056C000C03A0E94A7360E945C380E9423383F9659
:1056D0000E94C03A0E949039A0914903A530D1F5AB
:1056E000E3E70E945137EBE00E9456370E94C63A2A
:1056F000A83EE3E0BE0740F00E947B38BF010E9455
:10570000C63A0E944138EC930E94C63AA436E0E0C3
:10571000BE0740F00E94A038BF010E94C63A0E9416
:105720004C38EC930E94C63A1A9750F00E94AD385C
:10573000BF010E94C63A0E94A7360E945C38EC93D3
:105740000E945738BF010E94C63A0E949039EEE38A
:105750000E949D39A0914903A63059F5E8E70E94BF
:105760005137E0E00E94B73A0E94CB3AA436E0E01D
:10577000BE0740F00E947B38BF010E94CB3A0E94D6
:105780004C38EC930E94CB3A1A9750F00E94A03804
:10579000BF010E94CB3A0E94A7360E945C38EC936E
:1057A0000E94AD38BF010E94CB3A0E9490390E94FE
:1057B000D03AA0914903A73059F5E8E70E94513744
:1057C000E1E00E94B73A0E94D43AA436E0E0BE0776
:1057D00040F00E947B38BF010E94D43A0E944C38AE
:1057E000EC930E94D43A1A9750F00E94A038BF015F
:1057F0000E94D43A0E94A7360E945C38EC930E9423
:10580000AD38BF010E94D43A0E9490390E94D03A2C
:10581000A0914903A83059F5E8E70E945137E2E02A
:105820000E94B73A0E94D93AA436E0E0BE0740F0A1
:105830000E947B38BF010E94D93A0E944C38EC93F9
:105840000E94D93A1A9750F00E94A038BF010E94D6
:10585000D93A0E94A7360E945C38EC930E94AD387A
:10586000BF010E94D93A0E9490390E94D03AA0917B
:105870004903A93009F047C0ECE70E94933A0E941F
:105880006F31A031E7E2BE0738F00E946E380E9407
:105890006F310E94FE39EC930E946F31A83EE3E025
:1058A000BE0740F00E948038BF010E946F310E9405
:1058B0004138EC930E946F31A436E0E0BE0740F01F
:1058C0000E947B38BF010E946F310E944C38EC93DC
:1058D0000E946F311A9750F00E94A038BF010E94B9
:1058E0006F310E94A7360E945C38EC930E94AD385D
:1058F000BF010E946F310E949039E4E50E949839FF
:10590000E7E70E949D39AE81AF3571F50E947F3681
:10591000AFE8B3E00E94D231A091F603AA2342F48B
:10592000E0918F03F09190030E94C13D0E94E73700
:105930000E941938BF010E94EC370E9466390E940C
:105940007A3A0E94EC370E943C370E94F8370E9456
:105950009E3ABF010E94EC370E946B39EEE50E942F
:105960005239E1E00E945739AE81A03631F4E8E3C4
:105970000E94963AEDE00E945B37AE81A13631F489
:10598000E8E70E94143AEEE30E945B37AE81A2364C
:1059900061F4E8E30E945137FE01EE5BFF4F36965B
:1059A000A0913203A083E0E1E8ABAE81A33699F485
:1059B000E8E30E94963A0E94BE35EA17FB0718F406
:1059C000ECE00E945B370E94BE350E94C53519F09D
:1059D000EBE00E945B3731E0303108F089C00E9473
:1059E000E239EC91E03021F40E94E239EFE3EC93EC
:1059F0000E94E239AC91A63021F40E94E239EDE731
:105A0000EC930E94E239AC91A13021F40E94E2397A
:105A1000E6E0EC930E94E239AC91A23021F40E94BE
:105A2000E239EBE5EC930E94E239AC91A33021F42A
:105A30000E94E239EFE4EC930E94E239AC91A43089
:105A400021F40E94E239E6E6EC930E94E239AC913F
:105A5000A53021F40E94E239EDE6EC930E94E23990
:105A6000AC91A73021F40E94E239E7E0EC930E9468
:105A7000E239AC91A83021F40E94E239EFE7EC93CF
:105A80000E94E239AC91A93021F40E94E239EFE69C
:105A9000EC930E94E239AC91AA3021F40E94E239E1
:105AA000E0E0EC930E94E239AC91AB3021F40E942B
:105AB000E239E1E0EC930E94E239AC91AC3021F4A0
:105AC0000E94E239E8E0EC930E94E239AC91AD30FB
:105AD00021F40E94E239E0E4EC930E94E239AC91B7
:105AE000AE3021F40E94E239E9E0EC933F5F74CFDD
:105AF000E0910103E695E6950E94DE3A0E94E43AC1
:105B00000E94E93A0E94E43A0E94F13A0E94E43A83
:105B10000E94FC3A0E94E43A0E94A6390E94033B8C
:105B20000E94063B0E94033B0E940B3B0E94033BEA
:105B30000E94103BEAABE0910103E695E695E695FD
:105B40000E94DE3A0E94163B0E94E93A0E94163BF0
:105B50000E94F13A0E94163B0E94FC3A0E941B3BB5
:105B60000E94A6390E94203B0E94063B0E94203BD7
:105B70000E940B3B0E94203B0E94103BEBABE0914C
:105B80000103E6950E94DE3A0E941B3B0E94E93A1F
:105B90000E941B3B0E94F13A0E941B3B0E94FC3A70
:105BA0000E94163B0E94A6390E94233B0E94063B9E
:105BB0000E94233B0E940B3B0E94233B0E94103B10
:105BC000ECABFE01E65BFF4FE0810E94DE3A0E94F3
:105BD000263B0E94E93A0E94263B0E94F13A0E942D
:105BE000263B0E94FC3AE52F0E94A639EA2BAE2FF5
:105BF000E52F0E94063BEA2BAE2FE52F0E940B3BC0
:105C0000EA2BAE2FE0910103E170EA2BEDAB0E948D
:105C10002B3B0E94DE3A0E942B3B0E94303B0E94AD
:105C20002B3B0E94363B0E942B3B0E943F3B0E9435
:105C3000493B0E944D3B0E94503B0E944D3B0E94BD
:105C4000573B0E944D3BE295E170EA2BEEAB0E9480
:105C50005E3B0E94DE3A0E945E3B0E94303B0E9407
:105C60005E3B0E94363B0E945E3B0E943F3BE295BA
:105C70000E94A6390E94633B0E94503B0E94633BF6
:105C80000E94573B0E94633BE295E170EA2BEFAB29
:105C9000E52F0E946A3B0E945E3B0E94E93A0E9407
:105CA0005E3B0E94F13A0E945E3B0E94FC3A0E94D9
:105CB0006E3B0E94A6390E94733B0E94063B0E94E5
:105CC000733B0E940B3B0E94733B0E94103BE8AF6A
:105CD0000E94763B0E94DE3A0E94763B0E94303B57
:105CE0000E94763B0E94363B0E94763B0E943F3BDF
:105CF0000E947B3B0E94A6390E94733B0E94503B4E
:105D00000E94733B0E94573B0E94733BE295E170F7
:105D1000EA2BE9AF0E94803B0E94DE3A0E94803B62
:105D20000E94303B0E94803B0E94363B0E94803B99
:105D30000E943F3BEE1FE0E0EE1F0E94A6390E944A
:105D4000853B0E94503B0E94853B0E94573B0E942E
:105D5000853BE295E170EA2BEAAFE42FE2950E94E1
:105D6000DE3A0E94803B0E94E93A0E94803B0E94FA
:105D7000F13A0E94803B0E94FC3A0E94263B0E941E
:105D8000A6390E948C3B0E94063B0E948C3B0E94DD
:105D90000B3B0E948C3B0E94103BEBAF0E948F3B61
:105DA0000E94DE3A0E948F3B0E94303B0E948F3B54
:105DB0000E94363B0E948F3BE695E695E6950E9451
:105DC000943B0E2EA0E035FCA1E0EA2FEE0FEE0F83
:105DD000EE0FE0290E94993BE2950E949F3B0E94B2
:105DE000993B0E94573BEA2B0E94993BE295EF704A
:105DF000E695E170EA2BECAFFE01ED5BFF4FE08131
:105E0000E695E695E6950E94DE3AFE01ED5BFF4FD2
:105E1000E081E695E6950E94A43B0E94993B0E9492
:105E2000A83B0E94993B0E94943BAE2FE42F0E9416
:105E3000493BEA2BAE2FE42F0E94AF3BAE2FE42F5D
:105E40000E94B23BE42FE695E170EA2BEDAFE42F20
:105E50000E946A3B0E94B73BE2950E94A43BAE2F92
:105E60000E94B73B0E94F13A0E94B73B0E94BC3BA4
:105E7000AE2F0E94B73B0E94493BEA2BAE2F0E94F7
:105E8000B73B0E94AF3BAE2F0E94B73BE6950E9406
:105E9000B23B0E94B73BE170EA2BEEAFE42F0E94C9
:105EA0007B3B0E94DE3AE8A90E94A43BAE2FE8A902
:105EB0000E94A83BAE2FE8A9E695E6950E94943B88
:105EC000AE2FE0910103E2950E94A639EA2BAE2F96
:105ED000E42FEE1FE0E0EE1F0E949F3BAE2FE8A9EB
:105EE000E695E695E6950E94B23BE8A9E295E17059
:105EF000EA2BEFAFFE01F1963F960F01E8A90E9451
:105F00006A3B0E94C03BE2950E94A43BAE2F0E94D8
:105F1000C03B0E94F13A0E94C03B0E94BC3B0E94E1
:105F2000C53B0E94493BEA2B0E94C53B0E94AF3B08
:105F30000E94C53BE6950E94B23B0E94CB3BE170BC
:105F4000EA2BD001EC93FE01F19670960F01E8A9BF
:105F50000E947B3B0E94DE3A0E94CB3BE2950E946E
:105F6000A43B0E94C53B0E94F13A0E94CB3B0E9499
:105F7000BC3BAE2F0E94C03B0E94493BEA2BAE2F98
:105F80000E94C03B0E94AF3BAE2F0E94C03BE695F3
:105F90000E94B23B0E94C03BE170EA2BD001EC931F
:105FA00033FE0DC031E0313150F4E32FF0E0DE017B
:105FB000D196AE0FBF1FEFEFEC933F5FF4CF0E947F
:105FC000D03B3D3078F40E94D63BA2E5B8E00E9479
:105FD000D53DE17011F45D9801C05D9A0E94DD3BF2
:105FE0003F5FEFCF0E94E53B3D3078F40E94D63B07
:105FF000A0E3B8E00E94D53DE17011F45D9801C0C6
:106000005D9A0E94DD3B3F5FEFCF0E94E53B3D3054
:1060100078F40E94D63BA2E0B8E00E94D53DE17042
:1060200011F45D9801C05D9A0E94DD3B3F5FEFCFA8
:106030000E94E53B3D3078F40E94D63BA6E0B8E0F4
:106040000E94D53DE17011F45D9801C05D9A0E94F7
:10605000DD3B3F5FEFCF0E94E53B3D3058F50E94AE
:10606000EE3BA0913F030E94B433A0913E030E94F7
:10607000FC34A0E0F099A1E00E94783461F0ECE0FB
:10608000E31BA2E1B8E00E94D53DE17011F45D98F8
:1060900001C05D9A0BC0ECE0E31BA0E1B8E00E94F8
:1060A000D53DE17011F45D9801C05D9A0E94DD3B21
:1060B0003F5FD3CFA0913F030E94B433A0913E0332
:1060C0000E94FC34A0E0F099A1E00E94783419F01D
:1060D000E1E0E0933E03E0913F03E03019F4E0E0BB
:1060E000E0933E035D9A84E08A95F1F7289A84E074
:1060F0008A95F1F7289884E08A95F1F731E03A30F3
:1061000088F40E94EE3BE9E0E31BA0E4B1E00E94CA
:10611000D53DE17011F45D9801C05D9A0E94DD3BB0
:106120003F5FEDCF21E02131D8F431E03930B0F4D8
:106130000E94EE3BE22FF0E0DE01D196AE0FBF1FD2
:10614000AC91E8E0E31B0E94CD3DE17011F45D9855
:1061500001C05D9A0E94DD3B3F5FE8CF2F5FE3CF38
:106160005D9A85E28A95F1F7289A84E191E001979A
:10617000F1F70E94A533A92D0E94F33BAB2D0E949D
:10618000F33BAA2D0E94F33B0E94C0360E2A0E94C8
:106190001F35E0E0F0E060E07FEB0E94AB3D0E2AAF
:1061A0000E9477350E2A0E946E34E02929F0E0E043
:1061B000E0936B03E0936C03F09B03C0E0E0E0939B
:1061C0003F03A82DE4E60E941A3E0E2EA0E0F099AF
:1061D000A1E00E946B3329F00E940F33F09AE894FB
:1061E00033F80C94A906FFCFAA93E091C000E072A7
:1061F000E1F3E881E093C60021960895A09155034C
:10620000B09156030895A091C703B091C80380913F
:10621000C9039091CA030895E0E0F0E061EE75E4EF
:106220000E94463D0895E0916103F0916203089554
:10623000662777270E946E3C0E94313F0895E091C7
:106240006D03F0916E030895A091CF03B091D00338
:106250008091D1039091D2030895E0E0F0E060E2F4
:1062600071E40895A0916103B09162030895E0E0A4
:10627000F0E00E94433E0895A0916D03B0916E033B
:106280000895E091F703F091F8036091F90370919C
:10629000FA0308950E94353CED93FC930895A09174
:1062A000E303B091E4038091E5039091E603089540
:1062B000E0E0F0E06AE774E40E94F83CDF01CB0123
:1062C000ABCFA091DF03B091E0038091E103909107
:1062D000E2030895E0E0F0E060E070E00895A0914E
:1062E0007503B091760308950E94453F0E94A13C3A
:1062F0000895A0910704B091080480910904909139
:106300000A040895E0917B03F0917C0360917D0382
:1063100070917E030895A4E6B0E080E090E00E94D2
:10632000713EDF01CB01E091DF03F091E00360916A
:10633000E1037091E2030E94403F0895E0917303EE
:10634000F09174030895E0937303F0937403089538
:10635000A091FF03B0910004809101049091020488
:106360000895E093FF03F093000460930104709399
:1063700002040895A0917B03B0917C0380917D037A
:1063800090917E0308950E94713EDF01CB01E09160
:10639000FF03F091000460910104709102040E94D7
:1063A000403FA2CF0E94373CED93FC930895E0E07C
:1063B000F0E061EE75E40E94F83C0895A091E703D7
:1063C000B091E8038091E9039091EA030895E0E039
:1063D000F0EC69E774EC0E948B3D0895E7EEF3E082
:1063E000E0939103F09392030895E091E703F09115
:1063F000E8036091E9037091EA030895E091EB03EB
:10640000F091EC036091ED037091EE030895A0917B
:10641000CB03B091CC038091CD039091CE0308952E
:10642000E093CB03F093CC036093CD037093CE0342
:106430000895A091D303B091D4038091D503909196
:10644000D6030895E091CB03F091CC036091CD0386
:106450007091CE030895A091DB03B091DC0380918D
:10646000DD039091DE030895E0917703F0917803C6
:106470006091790370917A030895E0937703F09324
:1064800078036093790370937A030895EDDFE093C6
:106490006A04F0936B0460936C0470936D04089528
:1064A000A0917703B09178038091790390917A035A
:1064B0000895D3DE0E94F83C0895E0E00E941A3E61
:1064C0000E2E0895A091AB03B091AC038091AD0363
:1064D0009091AE0308950E22A0912703ECE30E9451
:1064E000153E0895A0916B03B0916C030895A0919F
:1064F0006903B0916A03BBCEE0916903F0916A032E
:106500000895A4E6B0E00C94F83BE7EAE0937A0043
:10651000A4E00C945C04EF2FF0E06E2EE7E2E09331
:106520007A000895E7EAE0937A00A3E00E945C0411
:10653000EF2FF0E09E2EE7E2E0937A000895E7EA7D
:10654000E0937A00A1E00E945C04EF2FF0E0BE2E01
:10655000E7E2E0937A000895EBE0E0937304E8EB60
:10656000E09374040895E0938103F0938203089507
:10657000E0938303F09384030895E0935903F09329
:106580005A0308956ADE0E94463D0895E0935F0332
:10659000F09360030895E0937B03F0937C03609392
:1065A0007D0370937E030895E0936903F0936A037B
:1065B0000895E0936F03F09370030895E093390317
:1065C000E0E0E09387040895E0917204F0E0E09346
:1065D0009903F0939A03E0917304F0E0EADFE0910D
:1065E0007404ECCFE0E0E0936E04E0936F04E0937A
:1065F0007004E0937104E0937204AECFE0E0E093A6
:106600007504E0937604E0937704E0937804E093D4
:1066100087040895E0939903F0939A030895AAE0FC
:10662000B0E00C94F83B0E945C040E94E23D0E94A2
:10663000DE3D0895E7EAE0937A00A0E00E945C0462
:10664000EF2FF0E00895E093AF03F093B003609371
:10665000B1037093B2030895E0915903F0915A0386
:106660000895E091AF03F091B0036091B103709190
:10667000B2030895E7E2E0937A008AE48A95F1F79D
:1066800008958AE48A95F1F7E7EAE0937A0008959D
:10669000A7E00E945C04EF2FF0E0E0934F03F0933B
:1066A00050030895A0914F03B09150030895E2E381
:1066B000F0E00E94433E0E2E0895A98DBA8DF7CFCB
:1066C000EEE1F0E00E943D3E0E2EA52DE1E00E949D
:1066D0001A3E0E220895E0E00E94F73DE021089561
:1066E000EAEFF0E00E94433E0E2EA52DE1E00E946D
:1066F0001A3E0E220895E4E00E94153EE02108951E
:10670000E0934F03F09350030895E0E0E0934F03CC
:10671000E09350030895E4E00E94F73D0E2E0895A3
:10672000A9A1E5E00E94F73D0895AA2DEAE00E94A4
:10673000153E0E2E0895A0E0F3FCA1E0E0E00E94DB
:10674000F73D0E22A02FE3E60895A62DEAE00E9471
:10675000153E0E2E0895B6DEE2E0F0E060E070E057
:106760000E94593EE0210895E1E00E94F73D0E2E7F
:106770000895A0911403AFCFE3E00E94F73D0E2EE1
:106780000895E0914F03F09150030895F297ADE71B
:10679000B0E00E94693E0F010895F0E0DE01979697
:1067A000AE0FBF1FEC91F0E0D0010E94A13EA8DF28
:1067B00079DFA93CE0E0BE070895EB85FC8572DF38
:1067C0000E94693EDF01E4E1F0E00E94A13E98CF23
:1067D000F0E0DE019B96AE0FBF1FEC91F0E062DFB0
:1067E0000E94693EDF01E4E6F0E00E94A13E88CF0E
:1067F000E12FF0E0DE019396AE0FBF1F0895A09148
:10680000A303B091A4038091A5039091A6030895DA
:10681000E8EEF3E060E070E00E94DE3EDF01CB01D5
:10682000B0DF662777270895EC91F0E0A0E4BCE99B
:106830000E94A13EE4DF662777270895E093A30333
:10684000F093A4036093A5037093A6030895D7DF84
:10685000DFCF0E94BC3DE5E0F0E060E070E00E9428
:10686000613E08950E94BC3DE4E1F0E060E070E02C
:106870000E94593E08950E94BC3DA431E0E0BE074D
:10688000E0E08E07E0E09E070895E091AB03F09111
:10689000AC036091AD037091AE03A0E5B4E180E07C
:1068A00090E00E949C3ECACFE8EEF3E060E070E02A
:1068B0000895A02FE3E60E94153E0895A0E0F0FCA5
:1068C000A1E009CFEFDEE0E0F0E00E941F3E089576
:1068D000E89425F8E0E0E09329030895E3DEC7CCCF
:1068E0000E22A0E022FCA1E0E1E00E94F73D089525
:1068F000E1E00E94F73DE0210895A0E025FCA1E041
:1069000033CFAF8DE3E00E94FC3DE0210895E0939A
:106910003603DECF0E2EA98DBA8DE0E0F0E00E94A6
:106920001F3E0E220895A0E021FCA1E0E0E00E94BD
:10693000F73D0895E0910403F0E03597B3DE0E943F
:106940003D3E0E2EE0913503BDDDFF2766277727FC
:106950000895A0E022FCA1E0BECEEB89FC89A091C5
:10696000AF03B091B0038091B1039091B203662759
:1069700077270E94593E0E2EEAE0F0E060E070E0DA
:106980000E94613E08956DDEAB89BC8988279927F6
:106990000E94BC3D0895A630E0E0BE07E0E08E070F
:1069A000E0E09E070895A0918103B09182030895CD
:1069B000E0918103F09182030895EB89FC89A09115
:1069C000AF03B091B0038091B1039091B2036627F9
:1069D00077270895EB85FC85A091F303B091F4032C
:1069E0008091F5039091F603662777270E946E3C0D
:1069F0000E94B13D0E2E0895E0E00E94F73D0E2268
:106A0000089550DEEAE00E94913E0895EB85FC85F2
:106A1000A091F303B091F4038091F5039091F603F4
:106A2000662777270E946E3C5FCCA0918303B091CC
:106A300084030895E0918303F09184030895A09165
:106A4000F303B091F4038091F5039091F603089558
:106A5000662777270E946E3C0895E091F303F0913A
:106A6000F4036091F5037091F603AB85BC8588272C
:106A700099270E94423F38CC0E94ED3D0E946E3C17
:106A80000895EAE0F0E00E94B43E3ACEE0911803A7
:106A900019DDFF27662777270895E0938B03F0938E
:106AA0008C030895E0911803F0E00CDD0E94ED3DA9
:106AB0000E94BC3D08950E94973EA0918B03B09127
:106AC0008C030895E0918B03F0918C030895A091BD
:106AD0001803BB27E091AB03F091AC036091AD03C9
:106AE0007091AE030E94F23D0E94BC3D0895A98DB5
:106AF000BA8DBDCBA0E0F099A1E0E1E00E94F73DA6
:106B0000EACC0E22A02FE3E60E94F73DE021089593
:106B10000E2EA0912703ECE30E94153E0E2208954D
:106B2000A1E0B0E00C94F83BE091DF03F091E003CA
:106B30006091E1037091E203ACE4B4E0ABCBFEDB27
:106B4000E0935604F0935704EBCFE0917503F09176
:106B500076030895EAE00E941A3E0E2E0895AB2DAA
:106B6000EAE00E94153E0E2EA0E027FCA1E044CFF3
:106B7000E0913203F0E0E05EFC4F0895ED85FE8584
:106B80000E94E23DA62DB0E008950E94373E0E2EF1
:106B9000A62DEAE00E941A3EE0210895A92DEAE020
:106BA0000E94153E0E2E0895E0910D03F0E0E85F7F
:106BB000FC4F0895E0915F03F09160030895A02FCA
:106BC000E3E60E94F73DE0210895E0913B03EF5F8B
:106BD000E0933B03E0913A03A0913B03EA17089549
:106BE000E0931903F0E048DFACE5BFE882E290E40F
:106BF0000E94F83CA3ECB5EF88E490E40E94F83CD6
:106C0000AFE5B3E047CB0E943D3E0E2EA0E023FC53
:106C1000A1E00895A0915F03B09160030895B6DCF0
:106C2000C9DF16DFDF01CB01ECE5FFE862E270E4CB
:106C30000E94463DDF01CB01E3ECF5EF68E470E430
:106C40000E94463DA9E1B3E00E94353CEC930895D3
:106C5000A0917303B09174030895E0912C03F0E0C8
:106C6000E65BFC4FA0810895A0912C03B0E0A65BE9
:106C7000BC4FEC910895A0913203B0E0A05EBC4FF0
:106C8000EC910895AE81E3E60E94F73D0E2E76CF9B
:106C9000E1E00E944E3FEA1B0E946C3F0895E091A4
:106CA0009903F0919A03A3EFB3E0E6DE0E94313F2F
:106CB0000895E093F303F093F4036093F503709366
:106CC000F6030895E091F303F091F4036091F50366
:106CD0007091F6030895A0919F03B091A0030895C9
:106CE000F1DFA0E0B0E080E09FE30895E093E303EC
:106CF000F093E4036093E5037093E60308959FDE49
:106D0000D8CBE0DFAFE8B3E04DCBEA1BFB0BB4DE42
:106D1000DF01CB01EAE9F9E969E271E40E94463D4D
:106D2000DF01CB01E0E0F0E068E571E4DDCAEE0FE1
:106D3000FF1FA0E0B4E00E944B3FE7CFE091C30308
:106D4000F091C4036091C5037091C6030895EAE011
:106D5000F0E00E94A13E0895A091C303B091C40346
:106D60008091C5039091C6030895CCDAD4CAE0930C
:106D7000BF03F093C0036093C1037093C2030895EF
:106D8000A1DBA8DA0E94613E0895EF85F889A09101
:106D9000AF03B091B0038091B1039091B203662725
:106DA00077270895A091AF03B091B0038091B1030C
:106DB0009091B2030895EA0FFB1FE0935D03F093F7
:106DC0005E0308950E94F430A0914F030C94F430B8
:106DD0000E94F430E0915E03AE2F0E94F430A09147
:106DE0005D030C94F430F0E0AE0FBF1FE0911B0385
:106DF000F0E00895F0E0AE0FBF1FE0914103F0E036
:106E0000AE0FBF1FE091420308950E94F430A0919D
:106E100016030E94F430A09117030C94F4300E94E2
:106E2000F430A0911B030C94F4300E94F430A09134
:106E30001C030C94F430A1E00E94F430A6E30C94FF
:106E4000F4300E94F430A0915D030C94F4300E9461
:106E5000F430A0E00E94F430A0E00895A091B303C4
:106E6000B091B4038091B5039091B6030895A091B9
:106E7000A103B091A2030895EAE0F0E00E94B43EBD
:106E80000895DE01AD5BBF4FEC930895EAE0DE01AB
:106E9000AB5BBF4FEC930895DE01AA5BBF4FEC9351
:106EA0000895DE01A95BBF4FEC930895DE01A85B56
:106EB000BF4FEC930895DE01A75BBF4FEC9308959D
:106EC000EAE0DE01A65BBF4FEC93DE01A55BBF4F9E
:106ED000EC93DE01A45BBF4FEC93DE01A35BBF4FDD
:106EE000EC93DE01A25BBF4FEC93DE01A15BBF4FD1
:106EF000EC93DE01A05BBF4FEC93DE01AF5ABF4FB6
:106F0000EC93089559E0E0913803E170EE0FAE2F55
:106F1000E0913803E695E170EE0FEE0FEE0FEA0F09
:106F20000E2E0895E0913803E695E695E170AE2FB8
:106F3000E0E0F5FCE1E0EA2BEE0FEE0FE00D4E2F66
:106F400008955E2FE0913803E170EE0FAE2FE091CF
:106F50003803E695E170EE0FEE0FEE0FEA0F0E2EFE
:106F6000E1CFE295E07FEE0FEE0F0895E0E020FC28
:106F7000E1E0E093010372CFAA30E0E0BE07E0E079
:106F80008E07E0E09E0708959DDAEAE0F0E060E019
:106F900070E008950E94DE3EDF01CB01EAE0F0E000
:106FA00060E070E00E94F83E0895FE01EE5BFF4F46
:106FB00034960895DE01AB5BBF4FEC930895E091EA
:106FC0008D03F0918E030E94C13DDF0155CFE09308
:106FD0008F03F09390030895A0918F03B0919003D5
:106FE0000895FE01EE5BFF4F3196BF01F5DF44CF00
:106FF000DF01EAE0F0E00E94E63EDB01EC93089559
:10700000FE01EE5BFF4F3296BF01E6DFEAE0F0E003
:107010000E94E63EDB01EC930895E0912C03A3E986
:10702000B3E0F0E0EE0FFF1FAE0FBF1F0E942D3F39
:107030000895FE01EE5BFF4F35960895E4E6F0E01B
:1070400060E070E00895EC93FE01EE5BFF4F089561
:1070500005DFEAE0F0E060E070E00895A0E020FCE9
:10706000A1E0EA2FE295E07F4E0F0895A09157032B
:10707000B09158030895FE01EE5BFF4F3D96BF01AE
:10708000F5CFE8EEF3E00E94A13EDF01EAE0F0E098
:107090000E94E33EDB010895E4E6F0E00E94A13E99
:1070A000DF01EAE0F0E00E94E33EDB010895FE012B
:1070B000EE5BFF4F3E960895DF01EAE0F0E00E94AC
:1070C000E33EDB0108950E94E33EDB01EC9308956B
:1070D000E2E0DE01A65BBF4FEC930895FE01EE5B9C
:1070E000FF4F3996BF010895BB27EAE0F0E00E9408
:1070F000E63EDB010895FE01EE5BFF4F3B960895EF
:10710000FE01EE5BFF4F3A9608950E94B93EDF0103
:10711000CB01EAE0F0E060E070E00E94F43E089508
:10712000A031E7E2BE07E0E08E07E0E09E070895A9
:10713000A83EE3E0BE07E0E08E07E0E09E0708958A
:10714000FE01EE5BFF4F3C960895A436E0E0BE07DB
:10715000E0E08E07E0E09E070895FE01EE5BFF4F42
:107160003D9608959DD9EAE0F0E060E070E0089572
:10717000FE01EE5BFF4F3F960895DE01A55BBF4F1A
:10718000EC93E4E7DE01A45BBF4FEC930895E0E4E9
:10719000DE01A05BBF4FEC930895DF01CB01E0E07F
:1071A000F0E060E171EC0E948B3D0895E0E4DE01C7
:1071B000A15BBF4FEC930895DF01CB01E0E0F0E06D
:1071C00066EC72EC0E948B3D0895E0E4DE01A25B68
:1071D000BF4FEC930895DF01CB01F9C8E0E4DE0175
:1071E000A35BBF4FEC930895A091B703B091B80390
:1071F0008091B9039091BA030895F6DFEAE0F0E0D8
:1072000060E070E00895E0918903F0918A030E94A4
:10721000C13DE0938903F0938A03089573D8A4E6EF
:10722000B0E080E090E0AFC8A0918903B0918A03FC
:107230000895BF01F9DFE0E1F7E20E94B43ED8CE45
:10724000BF01F2DFE8EEF3E00E94B43ED1CEBF0111
:10725000EBDFE4E6F0E00E94B43ECACEBF01E4DF1B
:10726000EAE0F0E00E94E63EDB01EC930895E0E501
:10727000DE01A35BBF4FEC930895A0919103B09101
:1072800092030895BF01F9DFE4E6F0E00E94B43E06
:10729000AFCEBF01F2DFEAE0F0E00E94E63EDB01A4
:1072A000EC930895DE01A55BBF4FEC930895DE01DA
:1072B000A45BBF4FEC930895DE01A35BBF4FEC933B
:1072C0000895E8EEF3E00E94B43E92CEE4E6F0E0EA
:1072D0000E94B43E8DCEEAE0F0E00E94E63EDB0183
:1072E000EC930895E98DFA8DF695E7950895E8EC0D
:1072F000F0E00E94A13EE0CEE4E1F0E00E94A13E79
:10730000DBCEE989FA89F695E7950895DE01A25B5F
:10731000BF4FEC930895A0916303B0916403089567
:10732000EAE0F0E0D0CEDE01A15BBF4FEC93089520
:10733000DE01A05BBF4FEC930895DE01AF5ABF4F53
:10734000EC9308950E942B3E0E2E91CDE170EE0F2E
:10735000EE0FEE0F0895ECE7AADF89CFA9A1E4E0D4
:107360000E94F73DAE2FE0E020FCE1E0EA23089523
:10737000AE2FE0E020FCE1E0EA230895ECE7D3DF64
:10738000E0E5D6CFE7E7CFDFE9E3D2CFF0E00E9438
:10739000313EEECFE4E10E941A3EE0210895E093F1
:1073A0002C03E8E77FCF83DFEAE086DFE9E7AEDFA3
:1073B000E0E5B9DFE0E5BCDFEAE0BFDFE1E0E09374
:1073C0003F030895E32FF0E0DE01AE5BBF4FAE0F49
:1073D000BF1F08950E94F73D0E2EAE8108950E94B2
:1073E000F73D0E2AAE810895AE81E2E30E94F73D9B
:1073F0000E2EAD89BE89E4EAF1E00895E0E1F7E2FE
:107400000E94A13E59CEBF01AD89BE89A0CC49DD05
:10741000E9E74CCDEDE645DDE3E748CDE9E341DDC5
:10742000E0E544DDEEE347CD3CDDE7E73FCDAE816F
:10743000E5E0D0CFE3E10E94F73DE0290895E72D94
:10744000F0E0DE019396AE0FBF1F0895A091A70351
:10745000B091A8038091A9039091AA030895EC919B
:10746000F0E0A0E4BCE90E94A13EF0DF66277727A8
:107470000895E093A703F093A8036093A903709382
:10748000AA030895E3DFC4C9E091AB03F091AC0314
:107490006091AD037091AE03A0E5B4E180E090E0AF
:1074A0000E949C3EE6CF7EDCEAE0F0E060E070E027
:1074B000089567D9F695E79523C9E8ABF3D8A436C4
:1074C000E0E0BE070895BF01EDD8E6CDFE01EE5B1A
:1074D000FF4F3696BF01E6D83ACCFE01EE5BFF4F78
:1074E0003796BF01DFD81CCF0E94F73D0E2EA0912A
:1074F0004203FEC9FE01EE5BFF4F3696BF010895C1
:10750000BF01A0917103B09172030895A0915B0334
:10751000B0915C030895E8E5C4DCE4E5C7CCEDE692
:10752000C0DCE8E3C3CCBDDCE0E5C0CCBADCEEE512
:10753000BDCCA0916703B09168030895FE01EE5B96
:10754000FF4F37960895E0E0EEDEE1E7F1DEE1E798
:10755000F4CEE3E7A6DCE4E7A9CCA0915103B09117
:1075600052030895A8DCF9CD9CDCECE79FCC9EDCAF
:10757000EBE0A1CCBF01A0915C04B0915D04089543
:10758000BF01A0915E04B0915F040895A0916004D2
:10759000B09161040895A0916204B09163040895CC
:1075A000E3E6C6DEE9E3C9CEA0916404B0916504C8
:1075B0000895A0916604B09167040895E170E7957D
:1075C000E0E0E795AE2F0895FE01E95BFF4FE08113
:1075D0000895E295EF70E695E170C3DCEA2BAE2FDB
:1075E0000895E295EF70E695E695E170E295E07F0B
:1075F000EE0FEA2BAE2F0895E295E170E295E07F61
:10760000EA2BAE2F0895EA2BAE2FDECFE695E17080
:10761000EE0FEE0F0895E695E695E170EE0F0895F2
:10762000E695E695E695E170EA2B0895FE01E85BA4
:10763000FF4FE0810895FE01E75BFF4FE081089571
:10764000EA2BAE2FF8CFEA2BAE2FF0CFFE01E55B91
:10765000FF4FE0810895FE01E15BFF4FE081089557
:10766000E695E1707EDCEA2BAE2F0895E695E6956F
:10767000E170E295E07FEE0FEA2BAE2F0895E695DC
:10768000E695E695E170E295E07FEA2BAE2FE52FD7
:107690000895E695E695E69559CEEA2BAE2FDBCF19
:1076A000E295EF70E695E170EE0FEE0F0895E2952A
:1076B000EF70E695E695E170EE0F0895FE01E25B4E
:1076C000FF4FE0810895EA2BAE2FFE01E05BFF4FF4
:1076D000E0810895E295EF70E69570CFFE01E35BDF
:1076E000FF4FE0810895EA2BAE2FF8CFFE01E05B5B
:1076F000FF4FE0810895E295EF70E695E6950895D5
:10770000FE01E45BFF4FE0810895EA2BAE2FFE01FE
:10771000EF5AFF4FE0810895EA2BAE2F97CFFE017D
:10772000EF5AFF4FE0810895E170E295E07FEA2B88
:107730000895AE2FFE01ED5BFF4FE0810895E170EB
:10774000EE0FEE0FEA2B0895E1700BDCEA2B0895A3
:10775000E695E170E295E07FEE0FEA2B0895E6955D
:10776000E695EDCFE170EE0FEA2BAE2F0895FE0106
:10777000EC5BFF4FE0810895E295EF70E695D4CF82
:10778000FE01EB5BFF4FE0810895AE2FFE01EA5B47
:10779000FF4FE0810895FE01EA5BFF4FE08108950D
:1077A000289885E28A95F1F731E008955E9884E0A3
:1077B0008A95F1F7ECE0E31B089584E08A95F1F7F0
:1077C0005E9A84E08A95F1F708955D9A85E28A953C
:1077D000F1F7289A85E28A95F1F7E2CF5E9884E086
:1077E0008A95F1F70895EAE00E94153E0E2A089561
:1077F000109639F08DEC9AE00197F1F7A895119762
:10780000C9F7089530976040704009F070580895A6
:10781000552342F4503811F4E0FF04C03196691F3B
:10782000791F6BF050E8572711F45F93CFC05F3F8B
:1078300031F0660F000C57956795752F08955F938B
:1078400000200AF0CFC0C8C050E8192E1522880FBA
:10785000991F9527550F879550E8072E0522660F2B
:10786000771F7527550F67950895689401C0E894B0
:107870005F93F2DF703818F07F3F08F4A7C056E13D
:10788000571BAAF4519558300EF4593030F0EFEFF1
:10789000FFEF6FEF7FE777F91AC077275523B9F02D
:1078A000EE0FFF1F661F771F5A95D1F710C077277D
:1078B000583028F0EF2FF62F672F5850F9CF552367
:1078C00031F076956795F795E7955A95D1F70020B1
:1078D0000AF45BD15F910895689401C0E8943097F1
:1078E00060407040B1F0002426F0772312F4009439
:1078F0004CD1172E7EE1112032F07A95EE0FFF1F4A
:10790000661F111CF9CFEF2FF62F612D5F938ADFD1
:107910005F9108954F93AF01FD01DA01AB01BC0106
:10792000CA01402D012C142E4F910895EA0FFB1F20
:10793000681F0895E095F0956095EF5FFF4F6F4FDA
:1079400008955F9381DF903871F150E8152604C0E7
:107950005F937ADF903839F1703821F1572F591B36
:107960002BF112F4D7DFFACF583118F0AA27BB2732
:107970008827583028F0AB2FB82F88275850F9CFD8
:10798000552329F08695B795A7955A95D9F7502D87
:10799000512572F0CBDF38F46795F795E79573952D
:1079A00013F420C0B7DF3EDF5F910895D8F7FBCF17
:1079B000EA1BFB0B680B51F010F40094BBDF66234D
:1079C00092F3EE0FFF1F661F7A95CBF7EE27FF2786
:1079D000662777275F910895EFEFFFEF6FE77FEF5F
:1079E0005F910895EFEFFFEF6FE77FE75F910895F5
:1079F0005F932ADF703851F3903841F301240894E3
:107A0000791F23F41CF300203AF3ECCF0F921F935D
:107A10002F933F934F93112722279927689FA00107
:107A20008F9F302D410D591F6B9F300D411D591FE8
:107A30008E9F27D0BF9F25D06A9F23D0BE9F1DD089
:107A4000AF9F1BD0AE9F110D291F391F491F591F12
:107A5000E32FF42F652F522F4F913F912F911F91BC
:107A60000F9066232AF0550FEE1FFF1F661F02C0FE
:107A700073954BF2CDDE5F910895100D211D391FD6
:107A800002C0200D311D491F591F08955F93DCDE90
:107A9000703821F411200AF49FCFA4CF903809F454
:107AA00095CF01240894970B1BF4D4F30020F3CF57
:107AB000792F1F932F933F934F9311241127222740
:107AC00033274427552790E2AE17BF0786074107A3
:107AD00030F0AE1BBF0B860B410B089401C088949D
:107AE000551F221F331F111CAA1FBB1F881F441FB5
:107AF0009A9551F7F901612D4F913F912F911F9167
:107B0000662332F0550FEE1FFF1F661F7A9543F272
:107B10007FDE5F91089599239AF0772342F09717BB
:107B200048F029F4AE17BF07860720F031F098948B
:107B300088940895989408940895189488940895C2
:107B40007723C2F7971798F3A9F7EA17FB07680797
:107B500088F399F3ECCFDFDFE1E009F008F0EE27DE
:107B60000895D9DFE1E009F008F4EE270895EA0F5F
:107B7000FB1F681F791F0895AE1BBF0B860B970B69
:107B80000895F195E195F0400895F0956095709510
:107B9000E195FF4F6F4F7F4F0895EE230E2EEA2F92
:107BA00019F0E6950A94E9F70895EE230E2EFD01EB
:107BB00021F0F695E7950A94E1F70895F695E79593
:107BC000F695E795F695E795F695E7950895FE2FD6
:107BD000FF0FFF0B6F2F7F2F08956F2F660F660B20
:107BE000762F08958B2F880F880B982F0895EA170A
:107BF000E1E009F0EE270895EA17E1E009F4EE2745
:107C00000895AE17E1E00CF4EE270895AE17E1E019
:107C10000CF0EE270895EA17E1E00CF0EE27089546
:107C2000AE17E1E008F4EE270895AE17E1E008F0A2
:107C3000EE270895EA17E1E008F0EE270895EA1725
:107C4000FB07E1E009F0EE270895EA17FB07E1E002
:107C500009F4EE270895AE17BF07E1E00CF0EE2718
:107C60000895EA17FB07E1E00CF0EE270895EA1704
:107C7000FB07E1E008F4EE270895AE17BF07E1E047
:107C800008F0EE270895EA17FB07E1E008F0EE2779
:107C90000895EA17FB0768077907E1E009F0EE2786
:107CA0000895EA17FB0768077907E1E00CF4EE276F
:107CB0000895AE17BF0786079707E1E00CF0EE279F
:107CC0000895EA17FB0768077907E1E00CF0EE2753
:107CD0000895FA9FF02DEB9FF00DEA9FE02DF10D36
:107CE00008957A9F702D6B9F700DF89F700DE99F1E
:107CF000700D6A9F602D710DFB9F600D711DE89FD7
:107D0000600D711D8827FA9FF02D610D781FEB9F84
:107D1000F00D611D781FEA9FE02DF10D681F781F9F
:107D200008956E2F6A9FF0016B9FF00D089574D037
:107D3000D0DF0EF426DF08957DD0D3DF0EF425DFEB
:107D400008950024112490E1AA0FBB1F001C111CF0
:107D50000E1A1F0A18F40E0E1F1E01C0A1609A957C
:107D600099F7FD01D001089557D0EBDF0EF409DF3C
:107D700008953F934F935F93002411244427552780
:107D800030E2AA0FBB1F881F991F001C111C441F43
:107D9000551F0E1A1F0A460B570B28F40E0E1F1EF6
:107DA000461F571F01C0A1603A9559F7FD01BC015C
:107DB000D001CA015F914F913F9108953BD0D9DF27
:107DC0000EF4E3DE0895BDDFFD010895E894B7FFEA
:107DD00004C0A095B09511966894F7FDD2DEB1DF8E
:107DE000FD010EF4CEDE0895C4DFFD01BC0108954F
:107DF000E89497FF09C0A095B09580959095AF5FE6
:107E0000BF4F8F4F9F4F689477FDBFDEB2DFFD01FC
:107E1000BC010EF4BADE0895E894F7FF02C0B1DEAB
:107E20006894B7FF06C0A095B095119600F803942A
:107E300000FA0895E89477FF02C0A7DE689497FFE0
:107E40000BC00024A095B095809590951196801D4B
:107E5000901D00F8039400FA0895ED91FC9111979C
:107E60000895ED93FD936D937C930895A881B98156
:107E70008A819B810895E883F9836A837B830895CF
:107E8000689401C0E89401D02ADD182E862F612D58
:107E9000192E972F712D1B2EBF2FF12D1A2EAE2FBD
:107EA000E12D089500240E160F0606060706089514
:107EB00000240A160B06089500240A160B0608066D
:107EC00009060895EA17FB07680779070895AE17B2
:107ED000BF07860797070895E894EE2309F0689492
:107EE0000895AC0FBD1F05900D928A95E1F7089596
:00000001FF
